:020000040800F2
:10000000C81B002069020008BB3A000885340008BC
:10001000713A0008890900089D43000800000000AB
:100020000000000000000000000000007D3B000810
:10003000F70A000800000000BF3A00087F3B0008F4
:10004000830200088302000883020008830200087C
:10005000830200088302000883020008830200086C
:10006000830200088302000883020008830200085C
:1000700083020008830200088D0900089D0900081A
:1000800083020008AD09000883020008830200080B
:10009000830200088302000883020008830200082C
:1000A000830200088302000883020008830200081C
:1000B000830200088302000883020008830200080C
:1000C00083020008830200088302000883020008FC
:1000D000830200085D4300086D4300087D4300086B
:1000E000F90A00088302000883020008830200085E
:1000F00083020008830200088302000883020008CC
:1001000083020008830200088302000883020008BB
:100110007D3D000883020008513C0008613C000856
:10012000BD0900088302000883020008830200085A
:10013000830200088302000883020008830200088B
:10014000830200088302000883020008830200087B
:1001500083020008CD090008DD0900088D4300086E
:10016000830200088302000883020008830200085B
:1001700083020008830200088302000800000000D8
:10018000830200088302000800F002F800F05CF827
:100190000AA090E8000C82448344AAF10107DA45E2
:1001A00001D100F051F8AFF2090EBAE80F0013F0D8
:1001B000010F18BFFB1A43F0010318471485000014
:1001C000348500000A444FF0000C10F8013B13F096
:1001D000070408BF10F8014B1D1108BF10F8015BA0
:1001E000641E05D010F8016B641E01F8016BF9D193
:1001F00013F0080F1EBF10F8014BAD1C0C1B09D1EA
:100200006D1E58BF01F801CBFAD505E014F8016B5B
:1002100001F8016B6D1EF9D59142D6D370470000ED
:100220000023002400250026103A28BF78C1FBD8FF
:10023000520728BF30C148BF0B6070471FB508F098
:1002400031FA1FBD10B510BD00F070F91146FFF76F
:10025000F5FF05F003FE00F08EF903B4FFF7F2FF9F
:1002600003BC04F049F900000948804709480047E9
:10027000FEE7FEE7FEE7FEE7FEE7FEE7FEE7FEE756
:10028000FEE7FEE704480549054A064B70470000B3
:100290003D3C000889010008C8150020C81B00204B
:1002A000C8170020C81700207047704753EA020C97
:1002B00000F069802DE9F04B4FF00006002B1FBFC6
:1002C000B3FA83F503FA05F424FA05F65E4012BF8B
:1002D0001643B2FA82F502FA05F4C5F120051EBFF5
:1002E00022FA05FC44EA0C04203556EA044C4FEA95
:1002F000144418BF641C4FF000084FF000099042EE
:1003000071EB030C39D3002919BFB1FA81F701FA57
:1003100007F6B0FA80F700FA07F6C7F120071EBF0C
:1003200020FA07FC46EA0C062037B6FBF4FCA7EBE4
:100330000507103F07F01F0BCBF120060CFA0BFB53
:100340002CFA06F644BFB3460026202FA4BF5E4613
:100350004FF0000B5BEA060C08BF4FF0010B19EBE6
:100360000B09ABFB027C48EB0608C01B06FB02CC6A
:100370000BFB03CC71EB0C01C1E70B460246414677
:100380004846BDE8F08B13B54FF000004FF0000178
:10039000AFF30080BDE81C40704710B54C1084EAF4
:1003A000530404D54042C1F1000138BF491E1B422D
:1003B00004D55242C3F1000338BF5B1EFFF776FF3E
:1003C00014F0804F04D04042C1F1000138BF491EF3
:1003D00014F0004F04D05242C3F1000338BF5B1E3B
:1003E00010BD032A40F2308010F0030C00F015809D
:1003F00011F8013BBCF1020F624498BF11F801CB28
:1004000000F8013B38BF11F8013BA2F1040298BF8C
:1004100000F801CB38BF00F8013B11F0030300F0F6
:100420002580083AC0F0088051F8043B083A51F89A
:1004300004CBA0E80810F5E7121D5CBF51F8043B9F
:1004400040F8043BAFF30080D20724BF11F8013B12
:1004500011F801CB48BF11F8012B24BF00F8013B74
:1004600000F801CB48BF00F8012B704710B5203AC7
:10047000C0F00B80B1E81850203AA0E81850B1E85D
:100480001850A0E81850BFF4F5AF5FEA027C24BF13
:10049000B1E81850A0E8185044BF18C918C0BDE80A
:1004A00010405FEA827C24BF51F8043B40F8043BD3
:1004B00008BF7047D20728BF31F8023B48BF11F888
:1004C000012B28BF20F8023B48BF00F8012B7047E2
:1004D0004FF0000200B5134694469646203922BFDD
:1004E000A0E80C50A0E80C50B1F12001BFF4F7AF28
:1004F000090728BFA0E80C5048BF0CC05DF804EB0A
:10050000890028BF40F8042B08BF704748BF20F877
:10051000022B11F0804F18BF00F8012B7047704775
:100520007047704700487047681500207546FFF710
:10053000F9FFAE4605006946534620F007008546A0
:1005400018B020B5FFF79EFEBDE820404FF0000632
:100550004FF000074FF000084FF0000B21F00701AB
:10056000AC46ACE8C009ACE8C009ACE8C009ACE8EE
:10057000C0098D46704710B50446AFF30080204691
:10058000BDE81040FFF769BE70B50546AC6B206C46
:1005900000F0500050BB206C40F4007020642068D4
:1005A000806800F04050E8B9207ED8B92068C06A61
:1005B00000F4700020B12068806800F4806088B981
:1005C0002068406820F0200021684860206C20F4FA
:1005D00080702064206C00F4805018B9206C40F0CA
:1005E00001002064204600F0D3FB0BE0206C00F0FB
:1005F000100018B1204600F0CDFB03E0A06BC16CE9
:100600002846884770BD70B50546AC6B4020206415
:10061000606C40F004006064204600F0BBFB70BDDD
:1006200070B50446A56B284600F0B3FB70BD000012
:1006300055494A6822F440324A604A6843681A437E
:100640004A600268526822F4807203685A60026845
:100650005368026943EA022203685A6002685268DA
:1006600022F0407203685A600268526883681A4335
:1006700003685A600268926822F4006203689A6014
:1006800002689268C3681A4303689A603F4B826AA3
:100690009A4218D00268926822F0706203689A60E9
:1006A00002689268836A1A4303689A6002689268D3
:1006B00022F0405203689A6002689268C36A1A4343
:1006C00003689A600BE00268926822F07062036827
:1006D0009A600268926822F0405203689A60026849
:1006E000926822F0020203689A6002689368027EB0
:1006F00043EA420203689A602022125CA2B10268B7
:10070000526842F4006203685A600268526822F438
:10071000604203685A6002685368426A521E43EAA4
:10072000423203685A6005E00268526822F40062AF
:1007300003685A600268D26A22F470020368DA62BF
:100740000268D36A828B521E43EA02520368DA625D
:100750000268926822F4007203689A6002689368E3
:1007600090F8302043EA422203689A600268926857
:1007700022F4806203689A6002689368426943EADF
:10078000822203689A607047002301400100000F35
:1007900030B52DED028B81B0044612E05848006858
:1007A000401C5749086008460068B0F5805F08DBC8
:1007B00000200860534890ED000B01B0BDEC028BA7
:1007C00030BD2021504800F0D5FF0028E6D1082C8C
:1007D0002DD2DFE804F004090E13181D222708218A
:1007E000012000F09BF822E01821012000F096F88B
:1007F0001DE02821012000F091F818E038210120A7
:1008000000F08CF813E04821012000F087F80EE09A
:100810005821012000F082F809E06821012000F051
:100820007DF804E07821012000F078F800BF00BFD7
:1008300000221021344800F0AFFFFC25284604F0C8
:100840003BFB0025284604F037FB0125284604F031
:1008500033FB0A2004F09CFE04F002FB8DF800003C
:1008600004F0FEFA8DF8010004F0FAFA8DF80200A7
:100870009DF8000000049DF8011040EA01209DF859
:1008800002100843214908600846006820490860B2
:100890000846006800F40000F8B108460068C0434C
:1008A000086008460068C0F3160008600846006843
:1008B000401C08600846006840420860084600681E
:1008C00007F09FFC41EC180B9FED120B53EC102B23
:1008D00007F000FD0B4A03C20DE00D48006807F069
:1008E00090FC41EC180B9FED0B0B53EC102B07F019
:1008F000F1FC044A03C2034890ED000B5DE70000E1
:1009000020000020180000200004024010000020F9
:100910001400002085F90F270088433F70B5044676
:100920000D4600221021164800F036FF0CE0154855
:100930000068401C1349086008460068B0F5805FF5
:1009400002DB0020086070BD20210D4800F012FF7E
:100950000028ECD104F00F0040F05006304604F0BF
:10096000ABFA0026304604F0A7FA284604F0A4FAB1
:1009700000221021024800F00FFF00BFE3E7000053
:10098000000402402000002000BFFEE710B502482E
:1009900000F0DCFB10BD00004C06002010B5024842
:1009A00000F0D4FB10BD00002C05002010B502485B
:1009B00000F0CCFB10BD0000EC05002010B5024893
:1009C00000F0C4FB10BD0000E001002010B502489B
:1009D00000F0BCFB10BD0000AC06002010B50248C2
:1009E00000F0B4FB10BD00008C0500200146087823
:1009F00010381823B0FBF3F20848805CC865032A5E
:100A000005D908686FF30900001D886503E00868D0
:100A10006FF309008865886D70470000AE86000896
:100A2000014600208A6A8B69CBB932B1012A0DD008
:100A3000022A03D0032A10D10EE000BFCB6A03F0D4
:100A40008073B3F1807F00D1012007E0CB6AB3F15E
:100A5000C07F00D1012001E000E000BF34E08B69DD
:100A6000B3F5005F1AD132B1012A07D0022A03D0B0
:100A7000032A11D10AE000BF01200EE0CB6A03F087
:100A80008073B3F1807F00D1012006E0CB6AB3F11F
:100A9000C07F00D1012000E000BF15E032B1012A83
:100AA00005D0022A04D0032A0CD103E000BF00BF06
:100AB000012008E0CB6A03F08073B3F1807F00D19E
:100AC000012000E000BF00BF704730B50468246813
:100AD00024F4802405682C60046863608468402CDA
:100AE00004D10468A2600468E16003E00468A160C6
:100AF0000468E26030BD704710B54FF4005000F05C
:100B000031FD10BD72B600BFFEE700000146084689
:100B1000024B33F8100002B290B2704786000020FA
:100B200001460846024B33F8100002B290B27047FB
:100B3000C809002030B5A0F11002D41702EB54749C
:100B4000E410094D2B5DD41702EB5474E410A2EBB2
:100B5000C4050124AC401C4014B101220A7001E01C
:100B600000220A7030BD00007A00002030B5024635
:100B7000D41702EB5474E410094D2B5D0246D417D0
:100B800002EB5474E410A2EBC4050124AC401C40F9
:100B900014B101220A7001E000220A7030BD000089
:100BA0007F00002010B51648002101600171082166
:100BB000302006F0D2FE022004F0DEFC092006F010
:100BC000BBFE0F49C8700A2006F0B6FE0C4908713A
:100BD0000921302006F0C1FE032004F0CDFC0620E0
:100BE00006F0AAFE06490870072006F0A5FE044993
:100BF0004870082006F0A0FE01498870084610BD24
:100C00006000002038B502460020009000BF92F836
:100C10003C00012801D1022038BD012082F83C00AF
:100C200000BF0868092816D91068C0680C780A3C0B
:100C300004EB44050724AC40A0431468E0600C7842
:100C40000A3C04EB44048868A0401468E46820432C
:100C50001468E06013E0106800690C7804EB440548
:100C60000724AC40A043146820610C7804EB4404D2
:100C70008868A0401468246920431468206148688B
:100C8000072817D21068406B0C79641E04EB8405AA
:100C90001F24AC40A04314686063088880B20C79BC
:100CA000641E04EB8404A0401468646B2043146841
:100CB000606331E048680D2817D21068006B0C792A
:100CC000E41F04EB84051F24AC40A0431468206398
:100CD000088880B20C79E41F04EB8404A0401468F7
:100CE000246B20431468206316E01068C06A0C79F6
:100CF0000D3C04EB84051F24AC40A0431468E06263
:100D0000088880B20C790D3C04EB8404A040146880
:100D1000E46A20431468E062194B1A4C1068A04240
:100D200006D10868122803D1586840F48000586042
:100D3000144C1068A0421CD10868102802D0086822
:100D4000112816D1586840F400005860086810282F
:100D50000FD10D4800680D4CB0FBF4F000EB8000A3
:100D60004000009002E00098401E0090009800288B
:100D7000F9D100BF002082F83C0000BF00BF4BE764
:100D800000230140002001400C00002040420F00E1
:100D9000704770477047000070B5044600250CB9D5
:100DA000012070BD1549A06A884200D000BF206CA8
:100DB00030B9204600F024F80020606484F83C003C
:100DC000206C00F0100088B9206C20F4885040F0AE
:100DD000020020642046FFF72BFC00206064206C9A
:100DE00020F0020040F00100206400E0012500BF77
:100DF000002084F83C0000BF2846D2E70100000F25
:100E000010B586B00446142101A8FFF761FB2849FC
:100E1000206888424AD100BF002000902548006821
:100E200040F48070234908600846006800F4807030
:100E3000009000BF00BF00BF002000901D48143884
:100E4000006840F004001B49143908600846006837
:100E500000F00400009000BF00BF012001900320BB
:100E600002900020039001A9134800F089FB134869
:100E70001349086000204860002111488160C1606A
:100E80004FF480610161490041618900816149112C
:100E9000C16100210162416200F078FA08B1FFF7F8
:100EA00031FE00BF0648A063846300BF06B010BDDA
:100EB0000020014044380240000802401064024013
:100EC000E0010020F8B504460D46164600200090CB
:100ED00000BF94F83C00012801D10220F8BD012098
:100EE00084F83C0000BF2068806800F00100A0B9D1
:100EF0002068806840F001002168886055480068DB
:100F00005549B0FBF1F000EB4000009002E0009882
:100F1000401E009000980028F9D12068806800F4F5
:100F20008070B0F5807F05D12068806820F48070E3
:100F3000216888602068806800F0010000287ED069
:100F4000206C40F20161884340F480702064206886
:100F5000406800F4806028B1206C20F4005040F418
:100F600080502064206C00F48050B0F5805F04D184
:100F7000606C20F00600606401E00020606400BF47
:100F8000002084F83C0000BF344F3548A16BC86393
:100F90003448A16B08643448A16BC8646FF0220028
:100FA000216808602068406840F0806021684860DF
:100FB0002068806840F4807021688860226802F1AF
:100FC0004C0133462A46A06B00F056FA786800F0D0
:100FD0001F0018BB25492068884213D02449206887
:100FE000884204D1381D006800F01F0050B121492B
:100FF000206888422BD11948001D006800F01F00AE
:10100000102824D22068806800F04050F8B9206889
:10101000806840F080402168886018E013492068AB
:10102000884214D12068806800F0405078B9206868
:10103000806840F080402168886008E0FFE7206C0D
:1010400040F010002064606C40F0010060640020FB
:1010500044E700000C00002040420F000023014044
:101060008905000821060008070600080020014045
:10107000002101400022014070B50446A56D00F03A
:1010800091FB064694F83500022808D08020606560
:1010900000BF002084F8340000BF012070BD20682C
:1010A000006820F01600216808602068406920F080
:1010B000800021684861206C08B9A06C28B12068C4
:1010C000006820F00800216808602068006820F0AF
:1010D00001002168086010E000F064FB801B052817
:1010E0000BD920206065032084F8350000BF002064
:1010F00084F8340000BF0320D0E72068006800F0C7
:1011000001000028E8D194F85C103F208840A860D6
:10111000012084F8350000BF002084F8340000BFAF
:1011200000BFBBE7014691F83500022803D08020BC
:10113000486501207047052081F83500086800687F
:1011400020F001000A6810600020F3E7F8B50446BB
:10115000002000908C4800684FF41651B0FBF1F766
:10116000A56D2E6894F85C1008208840304098B136
:101170002068006800F0040070B12068006820F06A
:1011800004002168086094F85C1008208840A8607A
:10119000606D40F00100606594F85C1001208840AB
:1011A000304068B12068406900F0800040B194F898
:1011B0005C1001208840A860606D40F0020060650E
:1011C00094F85C1004208840304068B120680068C2
:1011D00000F0020040B194F85C1004208840A86040
:1011E000606D40F00400606594F85C101020884049
:1011F000304078B32068006800F0080050B394F8DD
:101200005C1010208840A8602068006800F48020EE
:1012100080B12068006800F4002028B9206CC8B1B3
:101220002046216C884715E0A06C98B12046A16C3F
:1012300088470FE02068006800F4807028B92068B3
:10124000006820F0080021680860206C10B120467A
:10125000216C884794F85C1020208840304000289A
:1012600065D02068006800F0100000285FD094F876
:101270005C1020208840A86094F83500052828D10B
:101280002068006820F01600216808602068406926
:1012900020F0800021684861206C08B9A06C28B15A
:1012A0002068006820F008002168086094F85C104D
:1012B0003F208840A860012084F8350000BF00204E
:1012C00084F8340000BF206D10B12046216D88479E
:1012D000F8BD2068006800F4802080B120680068B4
:1012E00000F4002028B9606C10B12046616C88477A
:1012F0001DE0E06BD8B12046E16B884717E020681D
:10130000006800F4807068B92068006820F0100060
:1013100021680860012084F8350000BF002084F8AF
:10132000340000BFE06B10B12046E16B8847606D70
:1013300038B3606D00F00100F0B1052084F835008D
:101340002068006820F001002168086000BF009854
:10135000401C0090B84200D905E02068006800F009
:1013600001000028F3D100BF012084F8350000BF40
:10137000002084F8340000BFE06C10B12046E16C1E
:10138000884700BFA4E700000C0000202DE9F041D1
:101390000446002500F006FA074614B90120BDE80E
:1013A000F081606A00B100BF022084F8350000BF00
:1013B000002084F8340000BF2068006820F001009D
:1013C000216808600AE000F0EDF9C01B052805D986
:1013D00020206065032084F83500E0E7206800687D
:1013E00000F001000028EED1206805682148054082
:1013F000D4E901010843E1680843216908436169B0
:101400000843A1690843E1690843216A0843054389
:10141000606A042803D1D4E90B010843054320681E
:1014200005602068456925F00705606A0543606A24
:1014300004280DD1A06A0543E06A48B12046FFF7B1
:10144000EFFA28B140206065012084F83500A6E756
:10145000206845612046FFF7C9FA064694F85C10FB
:101460003F208840B06000206065012084F835008E
:10147000002094E73F8010F02DE9F04704460D4628
:1014800016461F464FF00008D4F8589000BF94F855
:101490003400012802D10220BDE8F087012084F841
:1014A000340000BF94F83500012825D1022084F8CB
:1014B0003500002060653B46324629462046FFF74E
:1014C00004FB94F85C103F208840C9F808002068AD
:1014D000006840F0160021680860206C28B1206880
:1014E000006840F00800216808602068006840F04B
:1014F00001002168086006E000BF002084F8340085
:1015000000BF4FF002084046C6E7000070B5044631
:1015100000F048F906462546681C10B104480078DA
:10152000054400BF00F03EF9801BA842FAD370BD0D
:1015300008000020B0F5005F10D109490978491C66
:10154000074A117011460978FF2901DA012100E0EC
:101550000021034A12785143014A1170704700007C
:101560005801002010B5044604480068204020B10E
:10157000024804602046FFF7DDFF10BD143C014027
:10158000F8B502460B460025002400200021D6E0D5
:10159000012606FA01F51E6806EA0504AC4274D17C
:1015A0001E7906F00306012E04D01E7906F003060C
:1015B000022E13D190684F000326BE40B0434F0067
:1015C000DE68BE4030439060506801268E40B043D4
:1015D0001E79C6F300168E40304350601E7906F027
:1015E0000306032E09D0D0684F000326BE40B04347
:1015F0004F009E68BE403043D0601E7906F003065F
:10160000022E13D1CF0802F1200656F827004E070C
:10161000F70E0F26BE40B0434F07FF0E1E69BE40B7
:101620003043CF0802F1200646F8270010684F002B
:101630000326BE40B0431E7906F003064F00BE40AD
:10164000304310605E6806F44036002E76D000BF4E
:10165000002600963C4E366846F480463A4F3E607F
:101660003E46366806F48046009600BF00BF374EFF
:101670008F0856F827008E07370F0F26BE40B0435D
:10168000334EB24202D1002624E057E0314EB2423E
:1016900001D101261EE0304EB24201D1022619E0EE
:1016A0002E4EB24201D1032614E02D4EB24201D19A
:1016B00004260FE02B4EB24201D105260AE02A4E45
:1016C000B24201D1062605E0284EB24201D10726DA
:1016D00000E008268F073F0FBE4030431B4E8F08A7
:1016E00046F82700224E3068A0435E6806F4801654
:1016F00006B120431E4E3060361D3068A0435E6840
:1017000006F4001606B12043194E361D3060184EFF
:10171000361F3068A0435E6806F4003606B12043E9
:10172000134E361F3060361F3068A0435E6806F4E3
:10173000803606B120430E4E083E3060491C102909
:10174000FFF426AFF8BD00004438024008380140DD
:10175000000002400004024000080240000C024069
:10176000001002400014024000180240001C024019
:10177000083C0140024613690B400BB1012000E018
:101780000020704710B5426921EA020302EA010411
:1017900043EA0443836110BD0AB1816101E00B0497
:1017A0008361704701480068704700000000002016
:1017B00070B504460CB9012070BD94F83D0028B9FD
:1017C000002084F83C00204600F0DAF8242084F859
:1017D0003D002068006820F0010021680860206852
:1017E000006840F40040216808602068006820F428
:1017F00000402168086000F0ADFA05465C49606869
:10180000884206D85B48854201D2012007E00020CB
:1018100005E05948854201D2012000E0002001285E
:1018200000D1C9E75548B5FBF0F62068406820F0C4
:101830003F003043216848604D496068884201D8C4
:10184000701C07E04FF4967070434FF47A71B0FB50
:10185000F1F0401C2168096A21F03F01084321682A
:10186000086243496068884214D8681E616849006C
:10187000B0FBF1F0401CC0F30B00042801D204209F
:101880003DE0681E61684900B0FBF1F0401CC0F308
:101890000B0034E0A06838B9681E616801EB4101B3
:1018A000B0FBF1F0401C0AE0681E616801EBC10268
:1018B00002EB0111B0FBF1F0401C40F48040C0F39A
:1018C0000B0008B901201AE0A06848B9681E6168D9
:1018D00001EB4101B0FBF1F0401CC0F30B000CE048
:1018E000681E616801EBC10202EB0111B0FBF1F06F
:1018F000401CC0F30B0040F4804040F400402168DD
:10190000C9694CF6FF72914308432168C861D4E964
:10191000070108432168096821F0C00108432168D4
:101920000860D4E9031008432168896848F2FF324F
:101930009143084321688860D4E905010843216880
:10194000C96821F0FF0108432168C8602068006869
:1019500040F001002168086000202064202084F805
:101960003D000020206384F83E0000BF24E7000013
:10197000A086010080841E0000093D0040420F0047
:1019800010B586B00446142101A8FEF7A1FD1B493D
:10199000206888422FD100BF0020009018480068BE
:1019A00040F00200164908600846006800F0020096
:1019B000009000BF00BFC0200190122002900020C4
:1019C0000390032004900420059001A90D48FFF71F
:1019D000D7FD00BF0020009009481030006840F497
:1019E00000100749103108600846006800F4001034
:1019F000009000BF00BF06B010BD000000540040C2
:101A00003038024000040240034800680349097866
:101A100008440149086070470000002008000020C9
:101A200010B50D48006840F400700B490860084686
:101A3000006840F4806008600846006840F48070E8
:101A40000860032000F0AAF8032000F007F800F077
:101A50002BF8002010BD0000003C024070B5044689
:101A60000E4800784FF47A71B1FBF0F00C49096828
:101A7000B1FBF0F5284600F0DBFC08B1012070BD99
:101A8000102C07D200222146501E00F049F80548CC
:101A9000046001E00120F2E70020F0E708000020E8
:101AA0000C0000200400002008B500BF00200090BA
:101AB0001048006840F480400E49086008460068FD
:101AC00000F48040009000BF00BF00BF00200090E5
:101AD000081F006840F08050091F08600846006831
:101AE00000F08050009000BF00BF052000F056F8C5
:101AF00008BD0000443802400146084600280DDBBE
:101B000000BF00BF00F01F0301229A4043099B0061
:101B100003F1E023C3F8002100BF00BF00BF7047FE
:101B20002DE9F05F80460D461646002702F0C8FCFE
:101B3000074639462A46334601F00700C0F1070A36
:101B4000BAF1040F02D94FF0040A01E0C0F1070A0C
:101B5000D14600F1040ABAF1070F02D24FF0000A91
:101B600001E0A0F1030AD4464FF0010A0AFA09FA8B
:101B7000AAF1010A0AEA020A0AFA0CFA4FF0010B6A
:101B80000BFA0CFBABF1010B0BEA030B4AEA0B045B
:101B90002146404602F09CFCBDE8F09F00BF00F0EB
:101BA0000702064B19684FF6FF031940044B0B431D
:101BB00043EA0221014B196000BF70470CED00E0C1
:101BC0000000FA0570B504460D460CB9012070BD41
:101BD0005848006800F00700A84209D255490D7026
:101BE0000846006800F00700A84201D00120EEE797
:101BF000207800F0020002281DD1207800F00400B7
:101C0000042805D14C48006840F4E0504A49086077
:101C1000207800F00800082805D14748006840F403
:101C20006040454908604448006820F0F000A16821
:101C3000084341490860207800F00100A8B36068BB
:101C4000012807D13C4808380068C0F34040B8B9C3
:101C50000120BCE76068022802D06068032807D131
:101C6000354808380068C0F3406048B90120AEE745
:101C7000314808380068C0F3400008B90120A6E7E1
:101C80002D48006820F00300616808432A49086075
:101C9000FFF788FD064609E0FFF784FD801B41F24F
:101CA0008831884202D9032091E707E02248006882
:101CB00000F00C006168B0EB810FEDD11D480068A9
:101CC00000F00700A84209D91A490D7008460068BB
:101CD00000F00700A84201D0012078E7207800F04A
:101CE0000400042807D11448006820F4E050E1689B
:101CF000084311490860207800F00800082808D13E
:101D00000D48006820F46040216940EAC1000A499A
:101D1000086000F03FF808490968C1F30311074A59
:101D2000515CC8400649086006480068FFF796FE07
:101D300000204CE7003C024008380240B68600080C
:101D40000C000020040000200148006870470000DB
:101D50000C00002000B5FFF7F7FF04490968C1F344
:101D60008221034A515CC84000BD0000083802408F
:101D7000C686000800B5FFF7E7FF04490968C1F30C
:101D80004231034A515CC84000BD0000083802409F
:101D9000C68600082DE9F047002400250026A1464C
:101DA0002548006800F00C0020B1042805D0082860
:101DB0003AD105E0DFF8849039E0DFF8849036E02E
:101DC0001D48001F006800F03F041B48001F00680A
:101DD00000F4800078B11A481749091F0968C1F357
:101DE0008811A0FB01700146224600233846FEF709
:101DF0005DFA05460EE011480F49091F0968C1F355
:101E00008811A0FB01700146224600233846FEF7E8
:101E10004DFA05460848001F0068C0F30140401C09
:101E20004600B5FBF6F902E0DFF8109000BF00BFF6
:101E30004846BDE8F0870000083802400024F4005E
:101E400000127A00F8B504460CB90120F8BD2078DC
:101E500000F00100002874D0F948006800F00C0080
:101E600004280DD0F648006800F00C00082813D1B3
:101E7000F348001F006800F48000B0F5800F0BD11C
:101E8000EF4808380068C0F34040002859D0606827
:101E9000002856D10120D9E700BF6068B0F5803F27
:101EA00008D1E7480838006840F48030E449083930
:101EB00008601EE06068B0F5A02F0DD1E04808383A
:101EC000006840F48020DE49083908600846006850
:101ED00040F4803008600CE0D9480838006820F4ED
:101EE0008030D749083908600846006820F480200F
:101EF000086000BF606890B1FFF754FC054606E03B
:101F0000FFF750FC401B642801D903209EE7CC4812
:101F100008380068C0F340400028F1D011E0FFF716
:101F200041FC054606E0FFF73DFC401B642801D953
:101F300003208BE7C24808380068C0F340400028FF
:101F4000F1D1207800F0020002285FD1BC4800687F
:101F500000F00C0058B1BA48006800F00C000828E6
:101F60001CD1B748001F006800F48000B0B9B44825
:101F700008380068C0F3400020B1E068012801D0B3
:101F8000012063E7AE480838006820F0F8002169B6
:101F900040EAC100AA490839086037E0E06800B3A8
:101FA0000120A8490860FFF7FDFB054606E0FFF7A2
:101FB000F9FB401B022801D9032047E7A048083855
:101FC0000068C0F340000028F1D09D480838006840
:101FD00020F0F800216940EAC100994908390860F9
:101FE00014E0002097490860FFF7DCFB054606E097
:101FF000FFF7D8FB401B022801D9032026E79048B1
:1020000008380068C0F340000028F1D1207800F0C3
:10201000080008282CD16069A8B101208A4908600D
:10202000FFF7C0FB054606E0FFF7BCFB401B02289C
:1020300001D903200AE782486C300068C0F34000F1
:102040000028F1D014E000207F490860FFF7AAFBC8
:10205000054606E0FFF7A6FB401B022801D9032036
:10206000F4E677486C300068C0F340000028F1D1F6
:10207000207800F00400042870D100277048383020
:10208000006800F0805090B900BF002000906C48BC
:102090003830006840F0805069493831086008469F
:1020A000006800F08050009000BF00BF0127674823
:1020B000006800F48070B0B96448006840F4807033
:1020C00062490860FFF76EFB054606E0FFF76AFB12
:1020D000401B022801D90320B8E65C48006800F4E0
:1020E00080700028F2D000BFA068012808D15448B1
:1020F0006830006840F001005149683108601DE017
:10210000A06805280DD14E486830006840F00400F2
:102110004B49683108600846006840F001000860DB
:102120000CE047486830006820F0010044496831FD
:1021300008600846006820F00400086000BFA0683E
:10214000A8B1FFF72FFB054609E0FFF72BFB401B6B
:1021500041F28831884202D9032077E626E03848E8
:1021600068300068C0F340000028EED013E0FFF7AD
:1021700019FB054608E0FFF715FB401B41F28831CB
:10218000884201D9032061E62D4868300068C0F319
:1021900040000028EFD1012F07D1294838300068CE
:1021A00020F0805026493831086000BFA06900281F
:1021B00045D02348006800F00C0008285DD0A069D5
:1021C000022845D100201F490866FFF7EBFA0546B3
:1021D00006E0FFF7E7FA401B022801D9032035E6A5
:1021E000174808380068C0F340600028F1D1D4E9EE
:1021F00007010843616A40EA81110122A06AC2EB2B
:10220000500041EA00412C20005D41EA00600C4989
:10221000091F086001200B490866FFF7C3FA05464D
:1022200006E0FFF7BFFA401B022801D903200DE6A4
:10223000034808380068C0F340600028F1D049E046
:102240000838024000004742800E474200700040BC
:10225000002021490866FFF7A5FA054606E0FFF7CA
:10226000A1FA401B022801D90320EFE51B480068B2
:10227000C0F340600028F2D12CE0A069012800D111
:10228000E4E51648001D0668A069012820D006F480
:102290008001E06981421BD106F03F01206A814242
:1022A00016D147F6C0703040616AB0EB811F0FD184
:1022B00006F440310122A06AC2EB5000B1EB004F9E
:1022C00006D106F070612C20005DB1EB006F01D0EB
:1022D0000120BBE50020B9E500004742003802407C
:1022E00010B504460CB9012010BD606A38B96068A9
:1022F000B0F5827F00D105E00021E16102E000211C
:10230000216161610021A16294F8510028B9002087
:1023100084F85000204600F047F8022084F851006D
:102320002068006820F0400021680860A08800F460
:102330008270218901F404410843A18901F40061FC
:102340000843217C01F002010843217D01F00101D5
:102350000843218B01F400710843217F01F038010B
:1023600008432021095D01F080010843218D01F41B
:1023700000510843216808600421A06901EA104067
:1023800094F8241001F01001084321684860206887
:10239000C06920F400602168C861002060650120E8
:1023A00084F8510000209FE710B586B00446142140
:1023B00001A8FEF78DF81B492068884230D100BF84
:1023C000002000901848006840F4804016490860DA
:1023D0000846006800F48040009000BF00BF00BFC6
:1023E0000020009010481038006840F002000E49AC
:1023F000103908600846006800F00200009000BF35
:1024000000BF4FF470400190022002900020039022
:10241000032004900520059001A90448FFF7B0F8B7
:1024200006B010BD003800404038024000040240B1
:1024300070B504462546681EB0F1807F01D30120A7
:102440000FE0681E4FF0E02148610F214FF0FF3090
:1024500002F03EF800204FF0E0218861072008617B
:10246000002070BD7047704730B502460B4600BF74
:1024700092F83C00012801D1022030BD012082F8F1
:102480003C0000BF022082F83D00106844681068DC
:10249000816824F070041868044310684460184D83
:1024A0001068A8421BD01068B0F1804F17D0154DAE
:1024B0001068A84213D0144D1068A8420FD0134DD5
:1024C0001068A8420BD0124D1068A84207D0114DD9
:1024D0001068A84203D0104D1068A84205D121F021
:1024E00080015868014310688160012082F83D0036
:1024F00000BF002082F83C0000BF00BFBDE7000025
:10250000000001400004004000080040000C0040B2
:1025100000040140004001400018004010B504468E
:102520000CB9012010BD94F83D0028B9002084F8B2
:102530003C00204600F026F8022084F83D00211DD2
:10254000206801F095FB012084F8460000BF84F864
:102550003E0001213F2001554020015541200155F9
:1025600000BF00BF012084F84200432001554420F1
:1025700001554520015500BF012084F83D00002091
:10258000D0E7000038B504461C492068884218D1BD
:1025900000BF002000901A48006840F01000184961
:1025A00008600846006800F01000009000BF00BFFF
:1025B000002211463620FFF7B3FA3620FFF79CFAC7
:1025C0001BE010492068884217D100BF002000900E
:1025D0000B48006840F02000094908600846006880
:1025E00000F02000009000BF00BF00220121372032
:1025F000FFF796FA3720FFF77FFA38BD001000404A
:102600004038024000140040014691F83D00012886
:1026100001D001207047022081F83D000868C068A1
:1026200040F001000B68D8601A4B086898421BD034
:102630000868B0F1804F17D0174B0868984213D044
:10264000164B086898420FD0154B086898420BD07B
:10265000144B0868984207D0134B0868984203D07F
:10266000124B086898420CD10868806800F0070295
:10267000062A0CD00868006840F001000B6818605A
:1026800005E00868006840F001000B681860002051
:10269000C0E70000000001400004004000080040C6
:1026A000000C0040000401400040014000180040C0
:1026B00001460868C06820F001000A68D06000BFC9
:1026C0000868006A41F21112104050B90868006AA7
:1026D0009210104028B90868006820F001000A68CC
:1026E000106000BF012081F83D00002070472DE9F7
:1026F000F04104460D4614B90120BDE8F08194F87C
:102700003D0028B9002084F83C00204600F054F831
:10271000022084F83D002068806844F20701884365
:1027200021688860211D206801F0A2FA2068D0F895
:102730000880206886692068076A286840EA0808D7
:1027400040F203308643A969A86840EA01200643A5
:1027500040F60C4086434FF2F0008643E969E86892
:1027600040EA0120064328690001296A40EA013055
:10277000064327F0220727F088076969686840EA5E
:10278000011007432068C0F808802068866120682F
:102790000762012084F8460084F83E0001213F20B2
:1027A0000155012084F8420043200155012084F89E
:1027B0003D000020A1E7000010B586B004461421BA
:1027C00001A8FDF785FE1B49206888422FD100BF74
:1027D000002000901848006840F001001649086089
:1027E0000846006800F00100009000BF00BF00BF75
:1027F0000020009010481438006840F010000E4986
:10280000143908600846006800F01000009000BF0E
:1028100000BF4FF42060019002200290002003903E
:1028200004900120059001A90448FEF7A9FE06B016
:1028300010BD00000000014044380240001002407A
:102840002DE9F04304460D4694F83E603F20075DB5
:1028500094F84280432010F804906DB9012E02D103
:10286000B8F1010F02D00120BDE8F083022084F806
:102870003E0084F8420025E0042D0CD1012F02D146
:10288000B9F1010F01D00120EEE702213F200155EF
:102890004320015516E0012E07D1012F05D1B8F1D3
:1028A000010F02D1B9F1010F01D00120DCE70220B4
:1028B00084F83E0002213F200155022084F84200A6
:1028C0004320015515B1042D0CD105E00122002152
:1028D000206801F041FA10E001220421206801F093
:1028E0003BFA0AE001220021206801F035FA0122BA
:1028F0000421206801F030FA00BF00BF20680068A2
:1029000040F00100216808600020ADE730B50446C2
:102910000D4615B1042D0CD105E0002211462068AA
:1029200001F01AFA10E000220421206801F014FAE4
:102930000AE000221146206801F00EFA002204216C
:10294000206801F009FA00BF00BF00BF2068006ADC
:1029500041F21111084050B92068006A89100840FE
:1029600028B92068006820F001002168086000BFD5
:102970000DB1042D28D11DB9012084F83E000EE0D0
:10298000042D03D101213F20015508E0082D03D17A
:1029900001214020015502E00121412001551DB9CE
:1029A000012084F842001AE0042D03D101214320C4
:1029B000015514E0082D03D10121442001550EE0FA
:1029C0000121452001550AE0012084F83E00012143
:1029D0003F200155012084F842004320015500208A
:1029E00030BD704770B504462068C5682068066928
:1029F00006F00200022819D105F00200022815D1C4
:102A0000401F21680861012020772068806900F05C
:102A1000030018B12046FFF7E4FF05E0204600F070
:102A200097F8204600F095F80020207706F0040083
:102A3000042819D105F00400042815D1C0432168E9
:102A40000861022020772068806900F4407018B186
:102A50002046FFF7C6FF05E0204600F079F8204643
:102A600000F077F80020207706F00800082819D138
:102A700005F00800082815D1C0432168086104202A
:102A800020772068C06900F0030018B12046FFF7E6
:102A9000A8FF05E0204600F05BF8204600F059F85A
:102AA0000020207706F01000102819D105F0100042
:102AB000102815D1C04321680861082020772068BC
:102AC000C06900F4407018B12046FFF78AFF05E0A6
:102AD000204600F03DF8204600F03BF8002020772B
:102AE00006F0010048B105F0010030B16FF00100BF
:102AF00021680861204600F02DF806F0800080284B
:102B000009D105F08000802805D1C0432168086103
:102B10002046FFF7A7FC06F04000402809D105F049
:102B20004000402805D1C04321680861204600F0DC
:102B300033F806F02000202809D105F020002028D5
:102B400005D1C043216808612046FFF78CFC70BDA9
:102B50007047704710B504460C48844201D104F018
:102B6000DBFD0B4884420FD16FF001000849096872
:102B700008610748FFF79CFD064880880549C88022
:102B80000020888003F07EFB10BD0000340300208D
:102B90007C0300208C1300207047704770470000B2
:102BA0002DE9F84F0446206805682068C66820684B
:102BB00047694FF00009CA4605F00F09B9F1000F47
:102BC0000AD105F0200038B106F0200020B12046DF
:102BD00001F09AF9BDE8F88FB9F1000F7CD007F049
:102BE000010018B906F49070002875D005F00100B6
:102BF00030B106F4807018B1606C40F00100606480
:102C000005F0040030B107F0010018B1606C40F02D
:102C10000200606405F0020030B107F0010018B155
:102C2000606C40F00400606405F0080048B106F0F4
:102C3000200010B907F0010018B1606C40F00800E6
:102C40006064606C002846D005F0200028B106F0D2
:102C5000200010B1204601F057F920684069C0F308
:102C6000801A606C00F0080010B9BAF1000F2DD086
:102C7000204601F0F0F82068406900F0400040284C
:102C800020D100BF00BF2168143151E8001F21F09E
:102C900040002168143141E80002002AF3D100BF4E
:102CA000E06B50B17748E16B0865E06BFEF73AFAEC
:102CB00088B1E06B016D88470DE02046FFF76EFF9D
:102CC00009E009E02046FFF769FF04E02046FFF72E
:102CD00065FF002060647DE7206B012878D105F056
:102CE0001000002874D006F010000028FAD000BFB1
:102CF00000200090206800680090206840680090E4
:102D000000BF00BF2068406900F04000402860D14B
:102D1000E06B006840681FFA80F8B8F1000F56D0E9
:102D2000A08D404553DDA4F82E80E06BC069B0F55E
:102D3000807F43D000BF00BF21680C3151E8001FE5
:102D400021F4807021680C3141E80002002AF3D19F
:102D500000BF00BF00BF2168143151E8001F21F0FF
:102D600001002168143141E80002002AF3D100BFBC
:102D700000BF00BF2168143151E8001F21F040005E
:102D80002168143141E80002002AF3D100BF20205D
:102D900084F842000020206300BF00BF21680C318E
:102DA00051E8001F21F0100021680C3141E80002B9
:102DB000002AF3D100BFE06BFEF75EF902206063EA
:102DC000A08DE28D801A81B22046FFF7E6FE01E772
:102DD00042E0A08DE18D401A1FFA80F8E08DD0B35B
:102DE000B8F1000F37D000BF00BF21680C3151E8A7
:102DF000001F21F4907021680C3141E80002002A84
:102E0000F3D100BF00BF00BF2168143151E8001F9B
:102E100021F001002168143141E80002002AF3D1B9
:102E200000BF202084F842000020206300BF00BFC4
:102E300021680C3151E8001F21F0100021680C318D
:102E400041E80002002AF3D100BF0220606341463E
:102E50002046FFF7A2FEBDE605F0800030B106F087
:102E6000800018B1204601F003FAB3E605F04000F7
:102E700030B106F0400018B1204601F022F8A9E672
:102E800000BFA7E68D3D000810B504460CB901202F
:102E900010BDA06900B100E000BF94F8410028B95E
:102EA000002084F84000204600F02AF8242084F80E
:102EB00041002068C06820F400502168C8602046A6
:102EC00001F0A0F82068006920F4904021680861B2
:102ED0002068406920F02A00216848612068C068A5
:102EE00040F400502168C86000206064202084F80D
:102EF000410084F842000020606300BFC8E7000082
:102F000010B586B00446142101A8FDF7E1FAE8499E
:102F10002068884256D100BF00200090E548006834
:102F200040F40020E34908600846006800F40020EF
:102F3000009000BF00BF00BF00200090DD481038A7
:102F4000006840F00100DB4910390860084600685D
:102F500000F00100009000BF00BF0320019002209C
:102F6000029000200390032004900820059001A9FE
:102F7000D148FEF705FBD148D14908604FF0006009
:102F800048604021CE4881600021C1604FF48061DB
:102F90000161002141618161C16101624162FEF70D
:102FA000F5F908B1FDF7AEFD00BFC548A063846325
:102FB00000BF022201213420FEF7B2FD3420FEF7CB
:102FC0009BFD73E1BF492068884259D100BF0020B2
:102FD0000090B848001D006840F01000B549091D78
:102FE00008600846006800F01000009000BF00BFB5
:102FF00000BF00200090AF481038006840F001008A
:10300000AC49103908600846006800F001000090E3
:1030100000BF00BF4FF4C06001900220029000206A
:103020000390032004900720059001A9A248FEF711
:10303000A7FAA548A54908604FF000604860402104
:10304000A24881600021C1604FF4806101610021CC
:1030500041618161C16101624162FEF797F908B186
:10306000FDF750FD00BF9948A063846300BF0122B3
:1030700011462520FEF754FD2520FEF73DFD15E104
:1030800093492068884257D100BF002000908948AA
:10309000006840F40030874908600846006800F482
:1030A0000030009000BF00BF00BF002000908148AA
:1030B0001038006840F001007E4910390860084669
:1030C000006800F00100009000BF00BF0C200190DC
:1030D0000220029000200390032004900720059016
:1030E00001A97548FEF74CFA7448303079490860F8
:1030F0004FF0006048604021764881600021C16047
:103100004FF480610161002141618161C16101620F
:103110004162FEF73BF908B1FDF7F4FC00BF6D48D2
:10312000A063846300BF022201212620FEF7F8FC81
:103130002620FEF7E1FCB9E067492068884258D1B3
:1031400000BF002000905B48006840F4802059498F
:1031500008600846006800F48020009000BF00BFAF
:1031600000BF0020009053481038006840F0020073
:103170005049103908600846006800F002000090CD
:1031800000BF00BF4FF44060019002200290002079
:103190000390032004900720059001A94F48FEF7F3
:1031A000EFF9464818384E4908604FF00060486013
:1031B00040214B4881600021C1604FF48061016172
:1031C000002141618161C16101624162FEF7DEF867
:1031D00008B1FDF797FC00BF4148A063846300BFBE
:1031E000022201212720FEF79BFC2720FEF784FC0A
:1031F0005CE03C492068884258D100BF0020009024
:103200002C48001D006840F020002A49091D086074
:103210000846006800F02000009000BF00BF00BF1B
:103220000020009023481038006840F00400214935
:10323000103908600846006800F00400009000BFE4
:1032400000BFC020019002200290002003900320C4
:1032500004900820059001A92348FEF791F91A4827
:103260001838224908604FF02060486040211F480C
:1032700081600021C1604FF48061016100214161E2
:103280008161C16101624162FEF780F808B1FDF71A
:1032900039FC00BF1548A063846300BF02220121EE
:1032A0004720FEF73DFC4720FEF726FC06B010BD88
:1032B000004C004040380240000002407060024074
:1032C0002C05002000100140B86402408C0500204D
:1032D00000440040EC05002000480040000402408B
:1032E0004C0600200014014000080240AC060020FB
:1032F00070B504460D46164694F8420020280BD1BE
:1033000005B10EB9012070BD002020633246294668
:10331000204600F08DFFF6E70220F4E710B50446E2
:1033200003492068884201D102F0F8FF10BD000077
:10333000001001402DE9F84F04460E461746994605
:103340004FF0000A94F84100202850D106B117B977
:103350000120BDE8F88F00206064212084F841003E
:10336000FEF720FA8246A784E784A068B0F5805F64
:1033700004D1206910B90025B04602E035464FF06F
:1033800000081EE05346002280212046CDF8009020
:1033900000F09EFF20B1202084F841000320D8E7F0
:1033A00045B9B8F80000C0F308002168486008F18A
:1033B000020803E02878216848606D1CE08C401EFC
:1033C000E084E08C0028DDD15346002240212046D5
:1033D000CDF8009000F07CFF20B1202084F841005F
:1033E0000320B6E7202084F841000020B1E7022046
:1033F000AFE70000F7B50446154694F841002028D1
:1034000036D1019800B10DB90120FEBD01982062AE
:10341000A584E58400206064212084F841001548DB
:10342000A16BC8631448A16B08641448A16BC864FD
:103430000020A16B086501AE23681A1D31682B4678
:10344000A06BFEF719F86FF040002168086000BF1C
:1034500000BF2168143151E8001F41F0800021684D
:10346000143141E80002002AF3D100BF0020CCE76C
:103470000220CAE7F13D0008493E0008A13D0008CE
:103480007047704700BFFEE71FB500200090019015
:10349000029003901548164908604FF48030486048
:1034A000002113488160016101210176002180F82B
:1034B0002010C1620F4981620021C1600121C161F8
:1034C00080F830104161FDF767FC08B1FDF71AFB89
:1034D0000A200090012001900320029069460448D0
:1034E000FDF790FB08B1FDF70DFB1FBD002001406B
:1034F000980100200100000F08B500BF00200090D7
:103500002648006840F480002449086008460068A6
:1035100000F48000009000BF00BF00BF00200090BA
:103520000846006840F4001008600846006800F48F
:103530000010009000BF00BF002211460E20FEF7D1
:10354000EFFA0E20FEF7D8FA002211460F20FEF700
:10355000E7FA0F20FEF7D0FA002211461120FEF7FD
:10356000DFFA1120FEF7C8FA002211463820FEF7D4
:10357000D7FA3820FEF7C0FA002211464520FEF7A0
:10358000CFFA4520FEF7B8FA002211464620FEF792
:10359000C7FA4620FEF7B0FA08BD000030380240F6
:1035A00000B587B0142102A8FCF792FF00BF0020ED
:1035B00001907E48006840F010007C490860084691
:1035C000006800F01000019000BF00BF00BF0020A5
:1035D00001900846006840F0040008600846006852
:1035E00000F00400019000BF00BF00BF0020019068
:1035F0000846006840F0800008600846006800F057
:103600008000019000BF00BF00BF0020019008466D
:10361000006840F0010008600846006800F0010002
:10362000019000BF00BF00BF002001900846006865
:1036300040F0020008600846006800F002000190B7
:1036400000BF00BF00BF002001900846006840F0A6
:10365000080008600846006800F00800019000BFFC
:1036600000BF002241F27F015148FEF795F8002289
:103670004EF202714F48FEF78FF8002248F64011D3
:103680004D48FEF789F8012241F610014948FEF73E
:1036900083F8012215214948FEF77EF801224CF2F9
:1036A00080014348FEF778F8002248F2712144482F
:1036B000FEF772F8012247F682014148FEF76CF8E6
:1036C00000224FF402713D48FEF766F84DF2FF000C
:1036D00002900120039000200490059002A9344834
:1036E000FDF74EFF4FF6127002900120039000206C
:1036F0000490059002A92F48FDF742FF41F2B00067
:10370000029000200390049002A92B48FDF738FF97
:1037100048F640100290012003900020049005908C
:1037200002A92548FDF72CFF40F21D200290012040
:10373000039000200490059002A92048FDF720FF87
:103740004FF4005002904FF4881003900020049032
:1037500002A91748FDF714FF40F20C500290002018
:103760000390049002A91648FDF70AFF4FF6F320D4
:1037700002900120039000200490059002A91048B7
:10378000FDF7FEFE4FF4907002900020039004902D
:1037900002A90A48FDF7F4FE002211462820FEF790
:1037A000BFF92820FEF7A8F907B000BD3038024065
:1037B00000100240000802400000024000040240E5
:1037C000000C024010B50B480B4908600B484860DC
:1037D000002109488160C1604FF4804101610021EE
:1037E00041618161C1610162FDF7E2FF08B1FDF74E
:1037F00089F910BD0054004040020020A08601005D
:1038000010B50E480E4908604FF4827048600021E0
:103810000B488160C160016141614FF48021816189
:103820000021C1610162416281620A21C162FEF729
:1038300057FD08B1FDF766F910BD000000380040E3
:103840009402002000B58BB0242102A8FCF740FEB2
:103850000020009001901848184908600120486035
:103860000021164881604FF6FF71C160002101619F
:1038700041618161032002900020039001200490A7
:1038800000200590069007900120089000200990E4
:103890000A9002A90948FEF72AFF08B1FDF732F99C
:1038A00000200090019069460448FEF7DDFD08B154
:1038B000FDF728F90BB000BD00000140EC0200202C
:1038C0001CB50020009001900E480F49086053205D
:1038D000486000210C48816040F2E731C16000215E
:1038E0008161FEF71BFE08B1FDF70CF90020009086
:1038F000019069460448FEF7B7FD08B1FDF702F9EB
:103900001CBD000000100040340300201CB5002046
:10391000009001900E480F49086053204860002134
:103920000C48816040F2E731C16000218161FEF7FF
:10393000F5FD08B1FDF7E6F800200090019069461A
:103940000448FEF791FD08B1FDF7DCF81CBD00004E
:10395000001400407C03002010B50B480B490860A0
:103960004FF4E1304860002108488160C160016186
:103970000C21416100218161C161FFF785FA08B125
:10398000FDF7C0F810BD0000004C0040C40300204B
:1039900010B50B480B4908604FF4E1304860002136
:1039A00008488160C16001610C2141610021816191
:1039B000C161FFF769FA08B1FDF7A4F810BD000076
:1039C000001001400C04002010B50B480B490860A2
:1039D0004FF4E1304860002108488160C160016116
:1039E0000C21416100218161C161FFF74DFA08B1ED
:1039F000FDF788F810BD000000440040540400208A
:103A000010B50B480B4908604FF4E13048600021C5
:103A100008488160C16001610C2141610021816120
:103A2000C161FFF731FA08B1FDF76CF810BD000075
:103A3000004800409C04002010B50B480B4908606A
:103A40004FF4E1304860002108488160C1600161A5
:103A50000C21416100218161C161FFF715FA08B1B4
:103A6000FDF750F810BD000000140140E4040020F0
:103A700000BFFEE730B502464FF6FF7012B10446B4
:103A8000A14200D130BD11E012F8014B604000238B
:103A90000AE000F0010424B140104AF20104604041
:103AA00000E040105C1CE3B2082BF2DB0C1EA1F11D
:103AB0000105A9B2E8D100BFE4E700BFFEE7704707
:103AC00070B50024002522E06006040E01221102D8
:103AD0001148FDF761FE0A2001F053FD4FF48051BB
:103AE0000D48FDF747FE10B144F0010401E024F059
:103AF00001040A2001F045FD00224FF480710648C0
:103B0000FDF74AFE0A2001F03CFD681CC5B2082DF5
:103B1000DADB204670BD00000000024070B50446AC
:103B2000002526E00A2001F02CFD04F0800028B1D9
:103B30000122D1021048FDF72FFE05E000224FF4CC
:103B400000610D48FDF728FE012211020A48FDF729
:103B500023FE0A2001F015FD6006040E00224FF43A
:103B600080710548FDF718FE0A2001F00AFD681C67
:103B7000C5B2082DD6DB70BD00000240704710B5FD
:103B8000FDF742FF10BD000000B593B0302107A83B
:103B9000FCF79EFC142102A8FCF79AFC00BF002051
:103BA00001902448006840F080502249086008468F
:103BB000006800F08050019000BF00BF00BF0020EF
:103BC00001901D48006840F480401B490860084689
:103BD000006800F48040019000BF00BF0120079002
:103BE0000004089002200D9041050E9104210F91D0
:103BF000A8211091022111910421129107A8FEF72A
:103C000021F908B1FCF77EFF0F20029002200390FB
:103C1000002004904FF4A05005904FF4805006907F
:103C2000052102A8FDF7CEFF08B1FCF76BFF13B02A
:103C300000BD0000403802400070004003480068AA
:103C400040F47000014908607047000088ED00E012
:103C500010B50248FEF7C6FE10BD00003403002078
:103C600010B50248FEF7BEFE10BD00007C03002028
:103C700010B502682D4B98420ED0B0F1804F0BD09A
:103C80002B4B984208D02B4B984205D02A4B984298
:103C900002D02A4B984203D122F070024B681A439B
:103CA000224B984220D0B0F1804F1DD0204B98423B
:103CB0001AD0204B984217D01F4B984214D01F4B5C
:103CC000984211D01E4B98420ED01E4B98420BD0FA
:103CD0001D4B984208D01D4B984205D01C4B984272
:103CE00002D01C4B984203D122F44072CB681A4395
:103CF00022F080034C6943EA040202608B68C362CD
:103D00000B688362094B984202D00C4B984201D158
:103D10000B69036301234361036903F001031BB1D2
:103D2000036923F00103036110BD0000000001409E
:103D30000004004000080040000C00400004014066
:103D4000004001400044014000480140001800408C
:103D5000001C00400020004030B501F01F05012488
:103D600004FA05F3046A9C430462046A01F01F0527
:103D700002FA05F52C43046230BD000010B502487C
:103D8000FEF70EFF10BD0000C403002070B505460D
:103D9000AC6B0020E085E0842046FEF7FFFE70BD9E
:103DA00070B506460025B46B20684069C0F3C015A5
:103DB00094F84100212805D125B10020E084204657
:103DC00000F08FF820684069C0F3801594F8420035
:103DD000222805D125B10020E085204600F03BF8DF
:103DE000606C40F0100060642046FEF7D7FE70BDA6
:103DF00070B50546AC6B2868006800F48070F8B9AF
:103E00000020E08400BF00BF2168143151E8001F8A
:103E100021F080002168143141E80002002AF3D12A
:103E200000BF00BF00BF21680C3151E8001F41F006
:103E3000400021680C3141E80002002AF3D102E081
:103E40002046FFF71DFB70BD70B50446A56B2846E4
:103E5000FFF717FB70BD00BF00BF02680C3252E8CD
:103E6000002F22F4907102680C3242E80013002BFC
:103E7000F3D100BF00BF00BF0268143252E8002F28
:103E800022F001010268143242E80013002BF3D142
:103E900000BF016B01290ED100BF00BF02680C32C8
:103EA00052E8002F22F0100102680C3242E80013A1
:103EB000002BF3D100BF202180F8421000210163C4
:103EC000704710B504462068C06820F040002168A3
:103ED000C860202084F841002046FFF7D1FA002076
:103EE00010BD00BF00BF02680C3252E8002F22F064
:103EF000C00102680C3242E80013002BF3D100BF6E
:103F0000202180F841107047F8B5044694F842002B
:103F1000222875D1A068B0F5805F0CD1206950B916
:103F20000025A66A20684068C0F308003080A06AB7
:103F3000801CA06215E0A56A0026A068B0F5805F2D
:103F400003D0A06828B9206918B920684068287093
:103F500004E02068406800F07F002870A06A401CE0
:103F6000A062E08D401E80B2E085002846D1206826
:103F7000C06820F020002168C8602068C06820F474
:103F800080702168C8602068406920F001002168C5
:103F90004861202084F8420000206063206B0128E3
:103FA00026D10020206300BF00BF21680C3151E8FA
:103FB000001F21F0100021680C3141E80002002AA6
:103FC000F3D100BF2068006800F0100010280AD16B
:103FD00000BF0020009020680068009020684068C2
:103FE000009000BF00BFA18D2046FEF7D6FD02E085
:103FF0002046FFF793F90020F8BD01E00020FBE721
:104000000220F9E72DE9F84F04462068006920F402
:104010004050E1680843216808612169A0680843AD
:1040200061690843E169084300902068C06849F26B
:104030000C618843009908432168C8602068406982
:1040400020F44070A16908432168486176492068DE
:10405000884203D075492068884203D1FDF78AFE63
:10406000814602E0FDF776FE8146E069B0F5004F3B
:104070006CD102206168A0FB015003461920A9FB06
:10408000007001462A463846FCF710F96421B0FB5F
:10409000F1F04FEA001A02206168A0FB01510B46C3
:1040A0001920A9FB00712A463846FCF7FFF8834621
:1040B00002206168A0FB015003461920A9FB007192
:1040C0002A463846FCF7F2F86421B0FBF1F000EB29
:1040D000C00101EB0010ABEB8000322101EBC0000E
:1040E0006421B0FBF1F000F0F8000AEB400A022076
:1040F0006168A0FB015003461920A9FB007001462E
:104100002A463846FCF7D2F8834602206168A0FBB5
:10411000015003461920A9FB00712A463846FCF7D6
:10412000C5F86421B0FBF1F000EBC00101EB001019
:10413000ABEB8000322101EBC0006421B0FBF1F059
:1041400000F007005044216888606AE0042061683C
:10415000A0FB015003461920A9FB007001462A4626
:104160003846FCF7A3F8824604206168A0FB0150A2
:1041700003461920A9FB007001462A463846FCF781
:1041800095F86421B0FBF1F000EBC00101EB0010E9
:10419000AAEB8000322101EB00106421B0FBF1F0AA
:1041A00000F0F00A04206168A0FB017003461920AA
:1041B000A9FB00513A462846FCF778F86421B0FB89
:1041C000F1F00AEB001A04206168A0FB01510B46D4
:1041D0001920A9FB00712A463846FCF767F8834688
:1041E00004206168A0FB015003461920A9FB007060
:1041F00001462A463846FCF759F86421B0FBF1F035
:1042000000EBC00101EB0010ABEB8000322101EBB1
:1042100000106421B0FBF1F000F00F005044216861
:104220008860BDE8F88F00000010014000140140D4
:1042300010B5034699629A85DA85002058642220D9
:1042400083F84200186928B11868C06840F480708B
:104250001C68E0601868406940F001001C686061FB
:104260001868C06840F020001C68E060002010BDA5
:10427000014691F84100212828D18868B0F5805F77
:104280000BD1086948B90A6A1088C0F308000B68A6
:104290005860086A801C086205E00B6A581C0862B6
:1042A00018780B685860C88C401E80B2C88458B912
:1042B0000868C06820F080000B68D8600868C06893
:1042C00040F040000B68D860002070470220FCE7F7
:1042D0002DE9F84304460D4617469846089E31E0FE
:1042E000701C70B3FDF75EFAA0EB0800B04200D876
:1042F00016B90320BDE8F8832068C06800F0040008
:10430000F8B1802D1ED0402D1CD020680068C0F36D
:10431000C000B0B100BF002000902068006800908D
:1043200020684068009000BF00BF2046FFF793FD63
:104330000820606400BF002084F8400000BF012016
:10434000D8E7FFE7206800682840A84201D1012093
:1043500000E00020B842C3D00020CBE710B50248EF
:10436000FEF71EFC10BD00000C04002010B5024832
:10437000FEF716FC10BD00005404002010B50248E2
:10438000FEF70EFC10BD00009C04002010B5024892
:10439000FEF706FC10BD0000E404002000BFFEE7AD
:1043A0000246024B23F812107047000086000020DE
:1043B00070B50A46B2F57F4F19D1A0F11001CC17A4
:1043C00001EB5474E410174D2C5D0B46DD1703EB25
:1043D0005575ED10A3EBC5060125B5402C43E5B29C
:1043E000CC1701EB5474E4100E4E355518E0BAB9F1
:1043F000A0F11001CC1701EB5474E410094D2C5DB1
:104400000B46DD1703EB5575ED10A3EBC506012533
:10441000B540AC43CD1701EB5575ED10014E745509
:1044200070BD00007A00002010B5012291030448FD
:10443000FDF7B2F9012251030148FDF7ADF910BDB6
:10444000000C024070B5002400224FF480411A484D
:10445000FDF7A2F9012001F09BF801229103164813
:10446000FDF79AF9012001F093F880211348FDF738
:1044700081F9012801D144F00104002518E064000D
:1044800000224FF400510C48FDF786F9012001F09D
:104490007FF8012251030848FDF77EF98021074883
:1044A000FDF768F9012801D144F00104681CC5B288
:1044B0000F2DE4DBA0B270BD000C024000000240F2
:1044C00002480068C0F30220704700000CED00E0D5
:1044D00010B5002804DB0A07130E054A135406E042
:1044E0000A07140E034A00F00F031B1FD45410BD1B
:1044F00000E400E018ED00E000BF7047B5EEC00A30
:10450000F1EE10FA02DBF0EE400A01E0F1EE400AB3
:10451000B0EE600A70470000024800880249088334
:1045200070470000E8000020C809002010B50122F3
:10453000024801680248FCF7C5FC10BDE8000020F5
:104540009801002010B52DED068BC848007830B1D9
:10455000012862D002287CD003285DD123E100F03D
:104560000FFAC349C14A127841F822000846BF49F0
:10457000097850F8210000EE100AB8EEC00AF0EEFB
:10458000040A20EE200ADFEDBB0A80EE201A9FED20
:10459000BA0A21EE000ABDEEC00A10EE100AB349B5
:1045A000097801EB8101B54A02EBC101B44A1268F6
:1045B00041F82200B2480068401CB1490860084632
:1045C0000068092801DD00200860002010E0A749EC
:1045D000097801EB8101A94A02EBC10151F82010D1
:1045E000CA17A84C18CCC9186241A64B06C3401C78
:1045F0000A28ECDB0A220023A24903C9FBF7CDFEFF
:10460000A149088200219F4A116051600120974909
:104610000870912000F0D6F924E100F0B1F9944936
:10462000924A127841F82200904A127851F82200FA
:1046300003F0E7FD41EC1A0B9FED940B53EC102BAC
:1046400003F02AFC41EC190B9FED920B53EC102B5D
:1046500000E049E003F03EFE41EC180B03F074FD6E
:104660008249097801EB8101844A02EBC1018B4A3E
:10467000126841F8220089480068401C8749086098
:1046800008460068092801DD00200860002010E0CD
:104690007649097801EB8101784A02EBC10151F8B2
:1046A0002010CA17774C18CCC9186241754B06C345
:1046B000401C0A28ECDB734903C903F0B9FD9FEDE8
:1046C000780B53EC102B03F0E7FB03F06DFD6E4904
:1046D000488200216B4A11605160022063490870D2
:1046E000A12000F06FF9BDE000F04AF960495F4A8F
:1046F000127841F8220008465C49097850F82100F8
:1047000000EE100AB8EEC00AF0EE040A60EE200ACD
:104710009FED581A80EE810ADFED570A20EE200A3D
:10472000BDEEC00A10EE100A5049097801EB810174
:10473000524A02EBC1015C4A126841F822005A4811
:104740000068401C5849086008460068092801DDD7
:1047500000200860002011E04449097801EB810144
:10476000464A02EBC10151F82010CA17454BD3E964
:10477000004309195A41434B06C3401C0A28EBDB8E
:104780000A2200233F4903C9FBF707FE3E498882FE
:1047900000213C4A11605160032034490870B12067
:1047A00000F010F95EE000F0EBF831492F4A127882
:1047B00041F822002D4A127851F8220003F021FD21
:1047C00041EC1A0B9FED310B53EC102B03F064FB03
:1047D00041EC190B9FED2F0B53EC102B03F07AFDDE
:1047E00041EC180B03F0B0FC2049097801EB810182
:1047F000224A02EBC101294A126841F822002B48E3
:104800000068401C2949086008460068092801DD45
:1048100000200860002010E01449097801EB8101B4
:10482000164A02EBC10151F82010CA17154C18CCDA
:10483000C9186241134B06C3401C0A28ECDB0A224C
:104840000023104903C9FBF7A8FD0F49C8820021C6
:104850000C4A11605160002004490870812000F06A
:10486000B1F800BF00BFBDEC068B10BD38000020C2
:104870000C0700200000004B00401C461C070020D5
:104880002800002040000020C8090020000000008F
:1048900000006041000000000088A3402C000020C0
:1048A0000000000000002440300000203400002000
:1048B0001FB581200390C02002904020019000206D
:1048C0000090002202211748FCF766FF062000F046
:1048D0008DF80A2000F050FE012202211148FCF759
:1048E0005BFF03AA0121002000F0BAF802AA01210F
:1048F000084600F0B5F801AA0121022000F0B0F846
:104900006A460121032000F0ABF80022022105488D
:10491000FCF742FF0A2000F02FFE082000F066F8A6
:104920001FBD0000000C024070B5002400220121D0
:104930001248FCF731FF00251BE0012211460F4809
:10494000FCF72AFF012000F023FE6006040E082178
:104950000A48FCF70FFF0443012000F019FE002273
:1049600001210648FCF718FF012000F011FE681C29
:10497000C5B2082DE1DB204670BD0000000C0240EE
:1049800010B5002202210E48FCF706FF102000F0AF
:104990002DF8FFF7C9FF0446FFF7C6FF40EA0424DD
:1049A000FFF7C2FF40EA042404F4000008B144F019
:1049B0007F44012202210248FCF7EEFE204610BD92
:1049C000000C024001B56A460121002000F048F8C1
:1049D000082000F00BF800BF04210348FCF7CAFED2
:1049E0000028F9D108BD0000000C024070B5044653
:1049F000002201211948FCF7CFFE002529E0012201
:104A000011461648FCF7C8FE012000F0C1FD04F075
:104A1000800028B1012210211048FCF7BDFE04E0FF
:104A2000002210210D48FCF7B7FE6006040E01209D
:104A300000F0AEFD002201210848FCF7ADFE012088
:104A400000F0A6FD08210548FCF794FE0443681C0D
:104A5000C5B2082DD3DB204670BD0000000C02401B
:104A60002DE9F04106460C461546002202210F486A
:104A7000FCF792FE0C2101EA8601621E02F003029D
:104A8000114341F04000FFF7B1FF002704E015F8A3
:104A9000010BFFF7ABFF7F1CA742F8DB01220221CD
:104AA0000248FCF779FEBDE8F0810000000C0240EE
:104AB00010B52DED0A8BCC480068082835D2DFE808
:104AC00000F004356697C8FCFAF90120FBF760FE98
:104AD000B0EE40CAF0EE60CA9FEDC40B53EC102B51
:104AE00051EC1C0B03F0F6FB41EC1B0B9FEDC10BD3
:104AF00053EC102B03F0D0F941EC1A0B9FEDBF0BD8
:104B000053EC102B03F0E4FC41EC190B9FEDBD0BB3
:104B100053EC102B03F0C0F941EC180B03F044FBED
:104B2000BA4908800120B049086059E10220FBF72A
:104B30002FFEB0EE40CAF0EE60CA9FEDAC0B53EC16
:104B4000102B51EC1C0B03F0C5FB41EC1B0B9FED34
:104B5000A90B53EC102B03F09FF941EC1A0B9FEDBE
:104B6000A70B53EC102B03F0B3FC41EC190B9FED9A
:104B7000A50B53EC102B03F08FF941EC180B03F04D
:104B800013FBA249488002209749086028E10320CE
:104B9000FBF7FEFDB0EE40CAF0EE60CA9FED930B4E
:104BA00053EC102B51EC1C0B03F094FB41EC1B0B52
:104BB0009FED900B53EC102B03F06EF941EC1A0BA8
:104BC0009FED8E0B53EC102B03F082FC41EC190B84
:104BD0009FED8C0B53EC102B03F05EF941EC180B9E
:104BE00003F0E2FA8949888003207F490860F7E0F2
:104BF0000420FBF7CDFDB0EE40CAF0EE60CA9FED99
:104C00007B0B53EC102B51EC1C0B03F063FB41ECC2
:104C10001B0B9FED780B53EC102B03F03DF941EC8F
:104C20001A0B9FED760B53EC102B03F051FC41EC6B
:104C3000190B9FED740B53EC102B03F02DF941EC85
:104C4000180B03F0B1FA7149C88004206649086066
:104C5000C6E00520FBF79CFDB0EE40CAF0EE60CA4E
:104C60009FED620B53EC102B51EC1C0B03F032FB4D
:104C700041EC1B0B9FED5F0B53EC102B03F00CF979
:104C800041EC1A0B9FED5D0B53EC102B03F020FC55
:104C900041EC190B9FED5B0B53EC102B03F0FCF870
:104CA00041EC180B03F080FA5849088105204E4961
:104CB000086095E063E031E0FFE70620FBF768FD60
:104CC000B0EE40CAF0EE60CA9FED480B53EC102BDB
:104CD00051EC1C0B03F0FEFA41EC1B0B9FED450B56
:104CE00053EC102B03F0D8F841EC1A0B9FED430B5B
:104CF00053EC102B03F0ECFB41EC190B9FED410B37
:104D000053EC102B03F0C8F841EC180B03F04CFAED
:104D10003E49488106203449086061E00720FBF7DE
:104D200037FDB0EE40CAF0EE60CA9FED300B53EC99
:104D3000102B51EC1C0B03F0CDFA41EC190B9FED3D
:104D40002D0B53EC102B03F0A7F841EC1B0B9FED40
:104D50002B0B53EC102B03F0BBFB41EC180B9FED1E
:104D6000290B53EC102B03F097F841EC1A0B03F0CE
:104D70001BFA2649888107201B49086030E0002083
:104D8000FBF706FDB0EE40CAF0EE60CA9FED170BD0
:104D900053EC102B51EC1C0B03F09CFA41EC1B0B59
:104DA0009FED140B53EC102B03F076F841EC1A0B2B
:104DB0009FED120B53EC102B03F08AFB41EC180B08
:104DC0009FED100B53EC102B03F066F841EC190B20
:104DD00003F0EAF90D49C88100200349086000BFCB
:104DE00000BFBDEC0A8B10BD2400002000000000B5
:104DF000000024403D0AD7A3703DEA3F00000000B8
:104E000000C06240AE47E17A14AEEF3FC80900200F
:104E100010B5002210211148FCF7BEFC0122082128
:104E20000E48FCF7B9FC06210020FBF777FD0821AE
:104E30000120FBF773FD00210220FBF76FFDA1218C
:104E40000320FBF76BFD00210420FBF767FD002228
:104E500010210248FCF7A0FC10BD00000004024035
:104E600070B50024002201211148FCF795FC0025B3
:104E700019E0012211460E48FCF78EFC012000F0DB
:104E800087FB6006040E4FF480710A48FCF772FC41
:104E90000443002201210648FCF77EFC012000F0BB
:104EA00077FB681CC5B2082DE3DB204670BD00000F
:104EB000001002400004024070B5044600220121A7
:104EC0001848FCF769FC002528E001221146154826
:104ED000FCF762FC012000F05BFB04F0800028B1CD
:104EE000012251021048FCF757FC05E000224FF464
:104EF00000710D48FCF750FC6006040E00220121F1
:104F00000848FCF749FC012000F042FB4FF4807197
:104F10000548FCF72FFC0443681CC5B2082DD4DB00
:104F2000204670BD001002400004024010B5A548A4
:104F3000008800EE100AB8EE400ADFEDA30A80EE0A
:104F4000201AA24890ED000AB4EE401AF1EE10FAD1
:104F50001ED09C48008800EE100AB8EE400ADFED33
:104F60009A0A80EE201A994880ED001A90ED000A06
:104F7000F3EE090AB4EEE00AF1EE10FA03DDB3EE47
:104F8000090A80ED000A914890ED000A00F0B4F99A
:104F90008C48408800EE100AB8EE400ADFED8A0A1D
:104FA00080EE201A8A4890ED000AB4EE401AF1EE25
:104FB00010FA12D08348408800EE100AB8EE400A7A
:104FC000DFED810A80EE201A814880ED001A8148C9
:104FD0007F4991ED000A02F047F87A48808800EE98
:104FE000100AB8EE400A9FED781AC0EE010A7A481E
:104FF00090ED000AF4EE400AF1EE10FA12D071487A
:10500000808800EE100AB8EE400ADFED6F0A80EEED
:10501000201A714880ED001A70486F4991ED000A1E
:1050200002F022F86E48C07800F04000402806D117
:105030006C480078052802D101206649087068484C
:10504000C07800F02000202806D1664800780528A6
:1050500002D10120614908706348006801287CD1B1
:105060000020614908606148C089A0F57A6000EEBF
:10507000100AB8EEC00ADFED5E0A80EE201A9FED3E
:105080005D0A21EE000A5C4880ED000A012021E063
:10509000C0F109014F4A121D02EB810191ED000A96
:1050A000C0F10A024B49091D01EB820181ED000AA2
:1050B000C0F10901494A121D02EB810191ED000A7C
:1050C000C0F10A024549091D01EB820181ED000A88
:1050D000411CC8B20A28DBDB3E4890ED0B0A80ED8C
:1050E000010A3E4890ED0B0A80ED010A3F48008C12
:1050F00000EE100AB8EE400A3F48D0ED000A30EE4C
:10510000600AF2EE040A80EE201A324880ED0B1A93
:1051100090ED0B0ADFED390A80EE201A9FED380A78
:1051200021EE000A80ED0C0A90ED0E0AD0ED0C0A7B
:1051300030EE600A80ED130A2C48408C00EE100A15
:10514000B8EE400A2C48D0ED000A30EE600AF2EECC
:10515000040A80EE201A214800E015E080ED0B1AC9
:10516000D0ED0B0A9FED251A80EE810ADFED240AAF
:1051700020EE200A80ED0C0A90ED0E0AD0ED0C0A0C
:1051800030EE600A80ED130A1E480068012818D12D
:1051900000201C4908601248007800F00300032832
:1051A0000FD10E480078012803D01749094801F0B3
:1051B000EBFD08480078012803D01449074801F0A6
:1051C000E3FD10BD8600002000007A446801002045
:1051D0006C010020A0130020700100203414002076
:1051E0007A0000207801002038010020C809002042
:1051F00000007A460000FA44740100200000614477
:105200000000C84240010020E014002024150020C6
:1052100010B50F48006801280AD100200C49086029
:1052200000F062FEFFF778F9FFF742FCFFF78AF91A
:105230000848006801280AD100200649086000F0EB
:10524000ADFA05490880084600880449C88410BDA5
:10525000F800002010010020EC000020C809002008
:1052600010B52DED028BB0EE408A00249FED0C0AA4
:1052700028EE000AB0EE408A9FED0A0A28EE000AE6
:10528000DFED090A80EE201ABCEEC10A10EE100A0A
:1052900084B20221204600F059F8BDEC028B10BD0B
:1052A0000000C8420000804500404E4510B52DED7D
:1052B000028BB0EE408A00249FED0C0A28EE000A13
:1052C000B0EE408A9FED0A0A28EE000ADFED090AD7
:1052D00080EE201ABCEEC10A10EE100A84B203213F
:1052E000204600F033F8BDEC028B10BD0000C84230
:1052F0000000804500404E4510B52DED028BB0EE0C
:10530000408A00249FED0D0A28EE000AB0EE408A84
:105310009FED0B0A28EE000ADFED0A0A80EE201A44
:10532000BCEEC10A10EE100A84B2074804600121E5
:10533000204600F00BF8BDEC028B10BD0000C84207
:105340000000804500404E45480000202DE9F04116
:1053500007460C464FF6FF7000EA8705C5F30D05BA
:10536000012C15D1012280214A48FCF715FA0122AF
:1053700040214848FCF710FA0A2000F002F9002208
:1053800080214448FCF708FA0A2000F0FAF82FE0E0
:10539000022C15D1012211033F48FCF7FDF901222F
:1053A00091023D48FCF7F8F90A2000F0EAF80022E3
:1053B000E1023948FCF7F0F90A2000F0E2F817E0C2
:1053C000032C15D10122D1023348FCF7E5F9012263
:1053D00091023148FCF7E0F90A2000F0D2F80022EF
:1053E0004FF400612C48FCF7D7F90A2000F0C9F807
:1053F00000263BE0012240212648FCF7CDF901229E
:1054000091022548FCF7C8F905F40040B0F5004FBB
:105410000AD1012220211F48FCF7BEF90122D10345
:105420001E48FCF7B9F90AE0002220211948FCF7D0
:10543000B3F900224FF400411848FCF7ADF90A20F7
:1054400000F09FF8002240211248FCF7A5F9002245
:105450004FF480611048FCF79FF90A2000F091F8A2
:105460004FF6FF7000EA4505701CC6B2102EC1DB76
:10547000012280210748FCF78FF901221103064819
:10548000FCF78AF90122D1020348FCF785F9BDE84F
:10549000F0810000000C02400008024000000240C1
:1054A00010B520480078092839D2DFE800F0380527
:1054B0000C131A20262C320000224FF480511A4877
:1054C000FCF76AF92BE000224FF400611648FCF764
:1054D00063F924E000224FF400411448FCF75CF922
:1054E0001DE0002280211148FCF756F917E0002248
:1054F00004210F48FCF750F911E0002201210C486B
:10550000FCF74AF90BE0012291030848FCF744F943
:1055100005E0012210210748FCF73EF900BF00BF5B
:1055200010BD00005C000020000C02400010024092
:10553000000402400008024010B5012280210C48FE
:10554000FCF72AF9012211030A48FCF725F9012288
:10555000D1020848FCF720F9002240210448FCF75A
:105560001BF900224FF480610248FCF715F910BDC9
:10557000000C02400008024001B50098FBF7C6FF8E
:1055800008BD00E000BF011EA0F10100FAD1704784
:1055900011B526E0009CB4F5617F02D94FF4617427
:1055A00000E0009C23464FF0E024A069A82404FBFF
:1055B0001301002908DB00BF4FF0E024A2698242FA
:1055C0000CDA8A42F8DA09E0084C214400BF4FF0B7
:1055D000E024A2698242FADD8A42F8DC009CE41AE7
:1055E0000094009C002CD5D118BD00004090020012
:1055F00010B500F021FC3F48007800F001020421C2
:105600003D48FCF7C9F83B480078C0F34002082148
:105610003948FCF7C1F837480078C0F38002102100
:105620003548FCF7B9F833480078C0F3C0022021B0
:105630003148FCF7B1F82F480078C0F30012402140
:105640002D48FCF7A9F82B480078C0F340124FF41E
:1056500000512A48FCF7A0F826480078C0F38012D1
:105660004FF480412548FCF797F822480078C2099A
:105670004FF400412148FCF78FF821480078214978
:1056800008701C4880781E4908701E480078097808
:1056900088420AD01749887800F0D2FA154948782C
:1056A00000F0CEFA00F034F805E01249487800F036
:1056B000C7FA00F02DF8FEF7C5FE000A124908707F
:1056C000FEF7C0FE1049487010211048FCF752F850
:1056D000044620210D48FCF74DF804EB40000A4930
:1056E00088700448C0780121B1EBD01F01D100F0CF
:1056F00033FA10BD7A00002000100240000802407A
:10570000EF000020EE0000207F000020000002409B
:1057100010B500224FF480710748FCF73DF80A20CD
:10572000FFF736FF012211020348FCF735F80A2083
:10573000FFF72EFF10BD00000008024010B5002446
:105740001548006820F00C001349086004E0601C54
:10575000C4B20120FFF71CFF02210F48FCF70AF832
:1057600008B1C82CF3DBC82C01DB012010BD0024DC
:1057700004E0601CC4B20120FFF70AFF02210648C2
:10578000FBF7F8FF08B9F02CF3DBF02C01DB01206C
:10579000ECE70020EAE70000000802402DE9F041B4
:1057A00000F0A4F800F082F8FFF7C8FFCC2000F06A
:1057B000A9F8BE2000F0A6F800F066F8074600F051
:1057C00063F80546072D05DDE843C5B2F843C7B2C7
:1057D000002600E001262C46200204B2E01904B2A3
:1057E00000EE104AB8EEC00AF6EE040A20EE200AD7
:1057F000BDEEC00A10EE100A04B216B12046BDE894
:10580000F081604200B2FAE710B50122022104489B
:10581000FBF7C2FF00F04AF8FFF790FF10BD000051
:105820000008024010B51748006820F00C00154928
:1058300008600846006840F0040008600022022169
:105840001048FBF7A9FF0220FFF7A2FE0122022168
:105850000C48FBF7A1FF0B48006820F00C00094939
:1058600008600C20FFF794FE02210648FBF782FF38
:1058700008B1012400E000243220FFF789FE204611
:1058800010BD00000008024070B50026012508E0A8
:10589000FFF7C8FF0446E00140EA6600C6B2681C94
:1058A000C5B2082DF4DD304670BD000010B50E48BD
:1058B000006820F00C000C4908600846006840F0C1
:1058C00004000860002202210748FBF765FF40F250
:1058D000EE20FFF75DFE012202210348FBF75CFF8B
:1058E0000F20FFF755FE10BD0008024010B5FFF76E
:1058F000DDFFFFF723FFCC2000F004F8442000F088
:1059000001F810BD70B504461B48006820F00C007B
:10591000194908600846006840F004000860012545
:1059200026E004F00106641086B10022022112482C
:10593000FBF732FF0220FFF72BFE012202210E4867
:10594000FBF72AFF3C20FFF723FE0FE00022022195
:105950000948FBF721FF3C20FFF71AFE0122022134
:105960000548FBF719FF0220FFF712FE681CC5B2BD
:10597000082DD6DD70BD00000008024000B587B0DC
:1059800000BF002001901048006840F002000E495E
:1059900008600846006800F00200019000BF00BFE8
:1059A0000022C0210948FBF7F7FEC0200290112019
:1059B0000390002004900320059002A90348FBF700
:1059C000DFFD07B000BD0000303802400004024097
:1059D0002DE9F04107460D46164600F0E7F9A020F4
:1059E00000F0BAF900F00CFA00B12CE0281200F037
:1059F000B3F900F005FA00B125E0E8B200F0ACF927
:105A000000F0FEF900B11EE000F0D0F9A12000F096
:105A1000A3F900F0F5F900B115E000240CE000F066
:105A200079F93855701EA04202D000F03FF901E02C
:105A300000F05CF9601C84B2B442F0DB00F0CEF9F7
:105A40000120BDE8F08100F0C9F90020F9E700006D
:105A500070B504460D4616460C2221460548FFF750
:105A6000B7FF044801682960416869608068A860E0
:105A700070BD0000D90700202DE9F0470746884691
:105A800091464646002533E015B106F01F0020BBC5
:105A900000F0A4F900240AE000F088F9A02000F04A
:105AA0005BF900F0ADF900B904E0601C84B2B4F514
:105AB0007A7FF1DB00BFB4F57A7F00D136E0301297
:105AC00000F04AF900F09CF900B12FE0F0B200F0CC
:105AD00043F900F095F900B128E0785D00F03CF959
:105AE00000F08EF900B121E0701C86B2681C85B20E
:105AF0004D45C9DB00F072F900240AE000F056F9C8
:105B0000A02000F029F900F07BF900B904E0601C46
:105B100084B2B4F57A7FF1DB00BFB4F57A7F00D1AF
:105B200004E000F05BF90120BDE8F08700F056F9D1
:105B30000020F9E770B504460D4616460548296869
:105B4000016069684160A96881600C222146FFF705
:105B500093FF70BDCD07002010B53C210E48FCF727
:105B6000D5FE49F218700C49096848623C210A4880
:105B7000FCF766FE002009490860094908600949E8
:105B800008609820084908600848C07800F07F0045
:105B90000649C87010BD0000EC02002088010020FA
:105BA0008C01002090010020940100207A00002048
:105BB0001C4800681C4908601C480068406A194974
:105BC00008600846006818490968401A1849884260
:105BD00005DA18480068401C164908600DE01148B5
:105BE000006811490968401A4CF25031884204DDBE
:105BF00010480068401E0F4908600E480068C0EB5E
:105C000000400849096808440B49086008460068D4
:105C10004FF6FF7101EA10400849088506480088E0
:105C2000488570478C01002088010020EC0200208C
:105C3000B03CFFFF9401002090010020C809002023
:105C400070B504462546002628E000224FF40041A6
:105C50001448FBF7A1FD05F0800028B10122402186
:105C60001148FBF799FD04E0002240210E48FBF7A4
:105C700093FD6806050E00224FF400410948FBF72A
:105C80008BFD0A20FFF784FC0122D1030548FBF7B6
:105C900083FD0A20FFF77CFC701CC6B2082ED4DB03
:105CA00070BD0000000C02400000024010B54FF42F
:105CB00000000949086000F011F84020064908601A
:105CC00000F00CF84FF480000349086000F006F87B
:105CD00080200149086010BD18040240002001E046
:105CE000411CC8B22828FBDB7047000010B580209B
:105CF00007490860FFF7F2FF402005490860FFF7F9
:105D0000EDFF4FF4800002490860FFF7E7FF10BD88
:105D10001804024070B50024002516E06006040E49
:105D200040200C490860FFF7D9FF0A48083800688E
:105D300000F0800008B1601CC4B24FF48000054937
:105D40000860FFF7CBFF681CC5B2082DE6DB2046D4
:105D500070BD00001804024070B5044600251FE025
:105D600004F0800018B180200F49086003E04FF470
:105D700000000D490860FFF7B1FF40200A490860A4
:105D8000FFF7ACFF4FF4800007490860072D01D1F1
:105D9000802008606006040EFFF7A0FF681CC5B2F3
:105DA000082DDDDB70BD00001804024010B5802016
:105DB0000949086040200860FFF790FF4FF4000099
:105DC00005490860FFF78AFF4FF480000249086028
:105DD000FFF784FF10BD00001804024010B54FF417
:105DE00000000649086040200860FFF777FF802028
:105DF00002490860FFF772FF10BD0000180402405E
:105E000010B580200B49086040200860FFF766FF4E
:105E100008480838006800F0800008B1012400E05C
:105E200000244FF4800003490860FFF757FF204625
:105E300010BD00001804024010B506480068012893
:105E400006D102210448FBF79DFC002001490860AF
:105E500010BD00002801002000100240FBF7E0FD0B
:105E6000FDF792FEFDF79CFBFDF746FBFDF70CFBF3
:105E7000FDF7A8FCFDF7C4FCFDF7E4FCFDF76CFDA5
:105E8000FDF786FDFDF7A0FDFDF7BAFDFDF7D4FD9A
:105E9000FDF716FDFDF73AFD1248FCF7B5FBFFF7DD
:105EA0005BFEFEF743FBFEF7B3FFFEF701FDFFF7D6
:105EB00043FB00F0EDF8FFF7A7FCFEF7B5FA00F0A2
:105EC00003FAFFF75BFD00F095FF00F075FD07E0BA
:105ED000FFF78EFBFFF79CF9FFF728F8FFF768FE46
:105EE000F6E700003403002010B52DED028B9FED86
:105EF0005C0AB0EE408AFAF755FE0446207859490C
:105F00000860084600680002086060780968084375
:105F1000544908600846006800020860A0780968D3
:105F200008435049086008460068B0F5000F0FDBD1
:105F300008460068A0F1807000EE100AB8EEC00AB2
:105F4000DFED490A80EE201A484880ED001A0BE088
:105F5000444890ED000AB8EEC00ADFED430A80EE37
:105F6000201A424880ED001A4048D0ED000A9FED0B
:105F7000400A9FED401A01EE200AF2EE080A80EE78
:105F8000201A3D4880ED001A90ED000AF2EE040A56
:105F900020EE200A39480078401E00EB8000384986
:105FA00001EB00103749097800EB810080ED000A11
:105FB00032480078401C31490870084600780328B0
:105FC0002FDD012251023048FBF7E6FB002026E0DE
:105FD0009FED230AB0EE408A00210EE000EB800224
:105FE000274B03EB021202EB810292ED000A30EE26
:105FF000080AB0EE408A4A1CD1B21429EEDBB3EE97
:10600000040AC8EE000ABCEEE00A10EE101A8AB2CA
:1060100000F10D011D4B23F81120411CC8B20628C8
:10602000D6DB1648007806280DDD012013490870DC
:1060300014480078401C134908700846007813285B
:1060400001DD002008700D480078042805DA0022E0
:106050004FF400710C48FBF79FFBBDEC028B10BDA9
:1060600000000000680000200000004B74000020C9
:1060700000A00C4600401C466C0000205C00002084
:10608000E80700207800002000080240C80900202E
:1060900010B501F00DFB00224FF400712A48FBF708
:1060A0007BFB0A20FFF768FA01202849087081214C
:1060B000002001F052FC0A20FFF75EFA022023497B
:1060C00008708121002001F048FC0A20FFF754FAF3
:1060D00003201E4908708121002001F03EFC0A20A7
:1060E000FFF74AFA012251021748FBF755FB0A2035
:1060F000FFF742FA0420154908708121002001F0C1
:106100002CFC0A20FFF738FA05201049087081217D
:10611000002001F022FC0A20FFF72EFA06200B498E
:1061200008708121002001F018FC0A20FFF724FAF2
:10613000012006490870002241020348FBF72CFBAE
:106140000A20FFF719FA10BD000802405C00002089
:106150002DE9F04104460D460CB1022D01DABDE8EF
:10616000F08126786778012E01D0002E48D1052FC6
:106170003AD008DC012F0DD0022F11D0032F15D0FB
:10618000042F37D118E0062F1CD00F2F20D0102F4E
:1061900030D123E0A81E81B2A01C01F033F82EE01C
:1061A000A81E81B2A01C01F0D5F828E0A81E81B27B
:1061B000A01C01F075F922E0A81E81B2A01C01F01C
:1061C000F5F91CE0A81E81B2A01C01F061FD16E0EB
:1061D000A81E81B2A01C01F0D1FB10E0A81E81B264
:1061E000A01C01F071FC0AE0A81E81B2A01C01F005
:1061F000EDFC04E06078012100F004F800BF00BF6E
:1062000000BFACE7F0B599B005460E460024002764
:1062100001222146641C0DF8012045F08002214630
:10622000641C0DF801202146641C0DF80160214614
:106230006846FDF71FFC0746FAB22146641C0DF8BC
:1062400001203A122146641C0DF801200B48008AF7
:10625000A04201DB204601E00848008A0749488245
:106260004A8AC8686946FAF7BCF80448428AC16895
:10627000034801F057FB19B0F0BD00008C1300205B
:106280000C0400202DE9F04100240E480568C48864
:10629000022C01DABDE8F081A01E295C601E285C9A
:1062A00041EA0027A01E81B22846FDF7E3FB06461F
:1062B000B74200D0EEE7034AD1881068FFF748FFE5
:1062C00000BFE7E78C13002010B50E480E490860A8
:1062D00000208880C88008720C48C8604FF4806035
:1062E000088200204882012209490A48FDF700F887
:1062F0006FF001000849096808610748FCF784F954
:1063000010BD00008C0A00208C1300208C0E002091
:106310005C0100200C0400207C03002010B518480C
:10632000808840F2FF3188420EDB002014498880CB
:1063300008460068002101604FF6FF730A2211A190
:106340001448FCF7F7FF14E0134801780C488288E2
:106350008088401C0A4B98801846006881540F487A
:10636000FCF7A6F900200D49096848620B48FCF7C4
:106370004BF9012208490748FCF7BAFF10BD00009D
:106380008C130020E695B0E68DAEE6BAA2E587BA9A
:10639000000000000C0400205C0100207C030020B1
:1063A00070B504460D46F9480078062874D2DFE837
:1063B00000F0033896FCFBFAF5480068401C40B931
:1063C000F4480068F24908602046B1EE000A00F087
:1063D0004BFEF0480068F049086008460068EC4948
:1063E0000968401A14281BDDEC48808C00EE100A66
:1063F000B8EE400AEA48D0ED000A30EE600AF2EE4C
:10640000040A80EE201A85ED0E1A4FF0FF30E049A5
:106410000860E1490860DD480078401CDB490870ED
:10642000ABE2DB480068401CA8BBDA480068D849EA
:106430000860D5ED0E0AB0EE001A80EE810A9FEDDD
:10644000D91AC0EE010A94ED110A94ED121A30EE39
:10645000411A94ED120A00EE810A85ED0F0A95EDBE
:106460000F0AD4ED110AB4EEE00AF1EE10FA02D2EE
:1064700095ED0F0A01E094ED110A85ED0F0A95EDF7
:106480000F0AD4ED120AB4EEE00AF1EE10FA04DDC0
:1064900095ED0F0A03E00BE06EE294ED120A85ED34
:1064A0000F0AD5ED0F0AB0EE600A204600F0DCFDC1
:1064B000B8480068B849086008460068B4490968E7
:1064C000401A0A280ADD4FF0FF30B1490860B2498E
:1064D0000860AE480078401CAC4908704DE295F861
:1064E000400005287CDAAA480068401C20B9A94869
:1064F0000068A749086021E095F8401005F1080000
:1065000000EB810090ED000AD4ED0B0AB4EEE00A36
:10651000F1EE10FA02D294ED0B0A07E095F8401064
:1065200005F1080000EB810090ED000A95F840109D
:1065300005F1080000EB810080ED000A9548006835
:10654000954908600846006891490968401A78280A
:1065500002DD04208D490870D5ED0E0AB0EE001A58
:1065600080EE810AD5ED010AB7EE001A70EE810ABD
:1065700020EE200AD4ED0B0AB4EEE00AF1EE10FA98
:106580003CDD8948007860BB95ED0F0AD5ED010A26
:10659000B7EE001A70EE810A20EE200A84ED100A90
:1065A00094ED100A02E0E6E1A2E1FFE0D4ED110A69
:1065B000B4EEE00AF1EE10FA02D294ED100A01E016
:1065C00094ED110A84ED100A94ED100AD4ED120A2C
:1065D000B4EEE00AF1EE10FA04DD94ED100A03E0E7
:1065E000B0E00BE094ED120A84ED100AD4ED100A2D
:1065F000B0EE600A204600F037FD1AE0D5ED0E0A35
:10660000B0EE001A80EE810AD5ED010AB7EE001A4D
:1066100070EE810A20EE200AD4ED0B0AB4EEE00AF7
:10662000F1EE10FA05D86048007810B901205E49F3
:106630000870D5ED0E0AB0EE001A80EE810AD5ED95
:10664000010AB7EE001A71EE600A20EE200AD4EDBE
:106650000B0AB4EEE00AF1EE10FA37D25248007895
:10666000012833D195ED0F0AD5ED010AB7EE001AD6
:1066700071EE600A20EE200A84ED100A94ED100AF3
:10668000D4ED110AB4EEE00AF1EE10FA02D294ED64
:10669000100A01E094ED110A84ED100A94ED100A3D
:1066A000D4ED120AB4EEE00AF1EE10FA02DD94ED38
:1066B000100A01E094ED120A84ED100AD4ED100ADC
:1066C000B0EE600A204600F0CFFC5EE0D5ED0E0A89
:1066D000B0EE001A80EE810AD5ED010AB7EE001A7D
:1066E00071EE600A20EE200AD4ED0B0AB4EEE00A47
:1066F000F1EE10FA49DB2C480078012845D1002042
:10670000294908702448006821490968401A4FF453
:10671000FA71484300EE100AB8EEC00A95F840102E
:1067200005F1200000EB810080ED000A4FF0FF3002
:10673000174908601849086095F84000401C85F822
:10674000400022E012480068401C18B91148006857
:106750000F4908600F4800680F4908600846006844
:106760000B490968401A06280FDD2046B1EE000AE1
:1067700000F07AFC4FF0FF300549086006490860D8
:1067800002480078401C01490870F6E078010020BA
:106790007C0100205001002080010020C809002059
:1067A000740100200000614484010020002019E0F1
:1067B00095ED070A05F1080101EB8001D1ED000A12
:1067C00030EE200A85ED070A95ED0D0A05F120014E
:1067D00001EB8001D1ED000A30EE200A85ED0D0AB3
:1067E000411CC8B20528E3DBD5ED0E0AB0EE001A55
:1067F00080EE810AD5ED010AB7EE001A70EE810A2B
:1068000020EE200AF1EE040A20EE200AD5ED070A58
:1068100080EE801A85ED071A95ED0D0AF1EE040A57
:1068200080EE201A85ED0D1A95ED070ADFED540A6A
:1068300020EE200A9FED531AC1EE000AB6EE000AC0
:1068400020EE800A84ED170A95ED0D0AF6EE000A97
:1068500020EE200ADFED4C0A80EE201A9FED4B0A55
:1068600021EE000A84ED180A95ED0D0ADFED480AC5
:1068700060EE200A9FED441A80EE810AF6EE000ACF
:1068800020EE200A84ED1D0A6078012802D002283B
:1068900026D112E094ED170A3E4880ED000A94EDEF
:1068A000180A80ED010A94ED1D0A80ED020A032208
:1068B00001460020FFF73EF913E094ED170A354832
:1068C00080ED000A94ED180A80ED010A94ED1D0A8E
:1068D00080ED020A032201460C20FFF72BF900E0AD
:1068E00000BF00BF2C480078401C2B49087044E0D2
:1068F0002A480068401C18B92948006827490860E0
:106900002748006827490860084600682349096845
:10691000401A0A282EDD6078012802D0022818D1FA
:106920000BE09FED210A214880ED000A2048C07845
:1069300000F0BF001E49C8700CE09FED1B0A1D4807
:1069400080ED000A1A48C07800F0DF001849C870CE
:1069500000E000BF00BF4FF0FF3010490860114950
:10696000086000F029F8002020700B480078401CD7
:106970000949087001E000E070BD00BF00BFFBE7FF
:10698000560E494090C2753E00007A440000C8424D
:106990008FC2F53DC8140020780100207C01002042
:1069A0005001002080010020000000006C01002048
:1069B0007A0000207001002000202949087000BFE3
:1069C00011E09FED280A2649083101EB800181ED95
:1069D000000A9FED240A2249203101EB800181ED5C
:1069E000000A411CC8B20528EBDB9FED1F0A1C48BA
:1069F00080ED010A9FED1B0A80ED0E0A9FED190A3A
:106A000080ED0F0A0020164981F8400017490870F0
:106A100000BF11E09FED130A1449083101EB80011A
:106A200081ED000A9FED0F0A1049203101EB800132
:106A300081ED000A411CC8B20528EBDB9FED0A0A74
:106A40000A4880ED010A9FED070A80ED0E0A9FEDCE
:106A5000050A80ED0F0A0020044981F840007047C4
:106A6000E0140020000000009A99193E241500202F
:106A700010B50446D4ED130AB0EE600AFDF73EFDF2
:106A8000D4ED150AB4EEE00AF1EE10FA7EDDD4ED95
:106A9000130AB0EE600AFDF731FDF2EE040AB4EE1F
:106AA000E00AF1EE10FA71D294ED1A0AD4ED1C0A44
:106AB000B4EEE00AF1EE10FA11DB94ED1A0AD4ED0F
:106AC0001B0AB4EEE00AF1EE10FA08D894ED1A0AA7
:106AD000D4ED130A30EE200A84ED1A0A0DE094ED8D
:106AE0001A0AB5EEC00AF1EE10FA02DD94ED1B0AA7
:106AF00001E094ED1C0A84ED1A0A94ED1E0AD4ED0F
:106B0000180A80EE201A94ED1A0A21EE000A84ED8C
:106B1000190AD4ED1D0A94ED1E1A80EE810AD4EDF7
:106B2000130A94ED141A70EEC10A20EE200A84EDC7
:106B30001F0A94ED130AD4ED190A30EE200AD4EDA1
:106B40001F0A30EE200AD4ED170A20EE200A84ED49
:106B5000200A94ED200A9FED891AC0EE010A94EDF7
:106B6000110A94ED121A30EE411A94ED100A00EE5B
:106B7000810A84ED100A94ED130A84ED140A94F846
:106B80008C00012822D194ED100A00E0EDE0D4ED54
:106B9000210AB4EEE00AF1EE10FA02D294ED100AE6
:106BA00001E094ED210A84ED100A94ED100AD4ED71
:106BB000220AB4EEE00AF1EE10FA02DD94ED100ABA
:106BC00001E094ED220A84ED100AA6E094F8580042
:106BD00010B101287CD144E094ED210A6848D0ED41
:106BE000000AB7EE001A71EE600A20EE200AD4ED1A
:106BF000100AB4EEE00AF1EE10FA02DD94ED100A8C
:106C00000AE094ED210A5E48D0ED000AB7EE001AC2
:106C100071EE600A20EE200A84ED100A94ED220A3B
:106C20005748D0ED000AB7EE001A71EE600A20EE68
:106C3000200AD4ED100AB4EEE00AF1EE10FA02D206
:106C400094ED100A0AE094ED220A4D48D0ED000AB6
:106C5000B7EE001A71EE600A20EE200A84ED100AE9
:106C600046E094ED210A4648D0ED000AB7EE001A3E
:106C700071EE600A20EE200AD4ED100AB4EEE00AAC
:106C8000F1EE10FA02DD94ED100A0AE094ED210A0B
:106C90003B48D0ED000AB7EE001A71EE600A20EE14
:106CA000200A84ED100A94ED220A3548D0ED000A3E
:106CB000B7EE001A71EE600A20EE200AD4ED100A39
:106CC000B4EEE00AF1EE10FA03D294ED100A0BE0F4
:106CD0000DE094ED220A2A48D0ED000AB7EE001A22
:106CE00071EE600A20EE200A84ED100A00E000BF79
:106CF00000BFD4ED010A94ED0A1A70EEC10AB0EE9D
:106D0000600AFDF7FBFBF2EE040AB4EEE00AF1EED6
:106D100010FA02D8012084F88C0094ED100AD4ED0A
:106D2000110AB4EEE00AF1EE10FA02D294ED100A64
:106D300001E094ED110A84ED100A94ED100AD4EDEF
:106D4000120AB4EEE00AF1EE10FA02DD94ED100A38
:106D500001E094ED120A84ED100AD4ED100AB0EEB1
:106D6000600AD4F89000804707E09FED060A84EDA2
:106D70001A0A9FED040A84ED190A10BD0000C842EA
:106D8000640100200000000070B505460C4628781C
:106D900020B101280ED0022825D11BE0207801283F
:106DA00004D1FFF709FE0520114908702846FFF7B6
:106DB0005FFE19E00E480078052806D1FFF7FCFDBC
:106DC0000120207000200A49087021462846FFF75C
:106DD000E7FA09E02078012804D1FFF7EDFD05204E
:106DE0000349087000E070BD00BF00BFFBE7000072
:106DF0007801002010B5032291490020FEF728FEFB
:106E000000209049087001204870002009E09FEDA3
:106E10008E0A8C49091D01EB800181ED000A411C9D
:106E2000C8B20A28F3DB9FED880A864880ED0B0A7A
:106E30009FED850A80ED0C0A9FED830A80ED0D0A17
:106E40009FED810A80ED0E0A9FED7F0A80ED0F0A0B
:106E50009FED7D0A80ED100AB1EE000A80ED120A66
:106E6000B3EE040A80ED110A9FED770A80ED130A54
:106E70009FED750A80ED140AB6EE000A80ED150A42
:106E80006F4890ED000A6F4880ED170A6C4890ED4E
:106E9000010AB5EEC00AF1EE10FA02D19FED6B0ABD
:106EA00002E0674890ED010A664880ED180A9FED00
:106EB000660A80ED190A9FED660A80ED1B0A9FEDB8
:106EC000650A80ED1C0A9FED600A80ED1A0A5C4895
:106ED00090ED020A5B4880ED1D0A9FED5F0A80ED90
:106EE0001E0A9FED590A80ED1F0A9FED570A80ED9B
:106EF000200A9FED550A80ED210A9FED530A80ED8F
:106F0000220A00204F4981F88C005448C1F89000B3
:106F10009FED4D0AD1F890008047032248490C208C
:106F2000FEF796FD00204E490870022048700020B0
:106F300009E09FED450A4A49091D01EB800181EDF9
:106F4000000A411CC8B20A28F3DB9FED3F0A4448FF
:106F500080ED0B0A9FED3C0A80ED0C0A9FED3A0A8A
:106F600080ED0D0A9FED380A80ED0E0A9FED360A7E
:106F700080ED0F0A9FED340A80ED100AB1EE000A91
:106F800080ED120AB3EE040A80ED110A9FED2E0A7D
:106F900080ED130A9FED2C0A80ED140AB6EE000A6C
:106FA00080ED150A264890ED000A2D4880ED170A5D
:106FB000234890ED010AB5EEC00AF1EE10FA02D1B5
:106FC0009FED220A02E01E4890ED010A244880ED60
:106FD000180A9FED1D0A80ED190A9FED1D0A80ED2C
:106FE0001B0A9FED1C0A80ED1C0A9FED170A80ED1D
:106FF0001A0A134890ED020A194880ED1D0A9FED08
:10700000160A80ED1E0A9FED100A80ED1F0A9FED03
:107010000E0A80ED200A9FED0C0A80ED210A9FEDFB
:107020000A0A80ED220A00200D4981F88C000D48E3
:10703000C1F890009FED040AD1F89000804710BD80
:10704000D4140020A0130020000000000024744984
:1070500000004842000048C2CDCC4C3D61520008BF
:1070600034140020AD52000810B52DED028BB0EEA7
:10707000408A044694ED110AB4EEC80AF1EE10FA03
:1070800002DDB0EE480A01E094ED110AB0EE408A4C
:1070900094ED120AB4EEC80AF1EE10FA02D2B0EE84
:1070A000480A01E094ED120AB0EE408A94ED110A0C
:1070B000D4ED120A30EE600AD4ED120A78EE600ABE
:1070C00080EE801A9FED4C0A21EE000A84ED0E0A34
:1070D00094ED0E0A9FED481AC0EE010A9FED470A93
:1070E00020EE800A84ED0D0A84ED0F8A94ED0F0ADC
:1070F0004348D0ED000AB7EE001A70EE810A20EE88
:10710000200A84ED210A94ED0F0AD0ED000AB7EEB3
:10711000001A71EE600A20EE200A84ED220A94ED36
:107120000F0AD4ED100AB4EEE00AF1EE10FA01DA1B
:10713000012000E0002084F8580094ED0F0A84ED4F
:10714000100A94F8580010B1012846D122E094EDBD
:10715000100A2B48D0ED000AB7EE001A71EE600A53
:1071600020EE200AD4ED120AB4EEE00AF1EE10FA95
:1071700002D894ED120A0AE094ED100A2048D0EDEE
:10718000000AB7EE001A71EE600A20EE200A84EDC4
:10719000100A23E094ED100A1948D0ED000AB7EE6A
:1071A000001A71EE600A20EE200AD4ED120AB4EE45
:1071B000E00AF1EE10FA02D894ED120A0AE094ED1A
:1071C000100A0F48D0ED000AB7EE001A71EE600AFF
:1071D00020EE200A84ED100A00E000BF00BF00206E
:1071E00084F88C00D4ED100AB0EE600AD4F8900058
:1071F0008047BDEC028B10BD0000C8420000614416
:10720000640100202DE9F04F9DB0054600240020C8
:10721000199064216846F9F75BF96878297840EAA3
:107220000129E878A97840EA0126012E01DA282E02
:107230007EDCB9F1370F7DDC06EB0900382879DCFC
:10724000F01DC11700EB5171C1F3C7011C91012260
:107250002046611CCCB20DF800202046611CCCB247
:107260000DF800202046621CD4B21C990DF80010C5
:107270000027BB462DE000200DF8040082461AE0EE
:1072800009EB070188B21BA9F9F754FC1DF80400AB
:107290009DF86C1001FA0AF10843C0B20DF8040021
:1072A000781C87B2B74202DB0120199006E00AF190
:1072B000010000F0FF0ABAF1080FE1DB00BF601C1B
:1072C000C4B21998012800D106E00BF1010000F0CA
:1072D000FF0B1C988345CEDB00BF21466846FCF7B8
:1072E000C9FB804608F0FF022046611CCCB20DF8B5
:1072F00000204FEA28222046611CCCB20DF8002065
:107300001248008AA04201DB204601E00F48008AB3
:107310000E4948824A8AC8686946F9F762F80B48FC
:10732000428AC1680A4800F0FDFA1DB0BDE8F08F3E
:1073300003E0FFE702201A9001E003201A900120E9
:107340001A99FEF75FFF00BFEFE700008C130020E3
:107350000C0400202DE9F04F9DB0054600240020CC
:1073600019906878297840EA0129E878A97840EAF4
:107370000126012E01DA312E7EDCB9F1300F7FDCDF
:1073800006EB090031287BDCF01DC11700EB5171C1
:10739000C1F3C7011C9101222046611CCCB20DF83B
:1073A000002002222046611CCCB20DF800202046AD
:1073B000621CD4B21C990DF800100027BB462DE0CA
:1073C00000200DF8040082461AE009EB070188B29C
:1073D0001BA9F9F7CBFB1DF804009DF86C1001FA0E
:1073E0000AF10843C0B20DF80400781C87B2B74216
:1073F00002DB0120199006E00AF1010000F0FF0A0B
:10740000BAF1080FE1DB00BF601CC4B21998012873
:1074100000D106E00BF1010000F0FF0B1C98834542
:10742000CEDB00BF21466846FCF724FB804608F00F
:10743000FF022046611CCCB20DF800204FEA282242
:107440002046611CCCB20DF800201348008AA042EF
:1074500001DB204601E01048008A0F4948824A8A31
:10746000C8686946F8F7BDFF0B48428AC1680B48F7
:1074700000F058FA1DB001E005E001E0BDE8F08F32
:1074800002201A9001E003201A9002201A99FEF7B8
:10749000B9FE00BFEEE700008C1300200C040020B2
:1074A0002DE9F04F99B00646002416B919B0BDE891
:1074B000F08F7078317840EA0127F078B17840EAAF
:1074C0000125012D65DB312D63DC302F5EDC781961
:1074D00000285BDB7819312858DC01222046611C2A
:1074E000CCB20DF8002003222046611CCCB20DF86E
:1074F00000206806020E2046611CCCB20DF8002068
:107500004FF0000817E007EB080188B2F9F7FEFA20
:1075100081464FEA29222046611CCCB20DF800209A
:1075200009F0FF022046611CCCB20DF8002008F1E2
:1075300001001FFA80F8A845E5DB21466846FCF704
:1075400099FA82460AF0FF022046611CCCB20DF87F
:1075500000204FEA2A222046611CCCB20DF8002000
:107560001048008AA04201DB204601E00D48008A55
:107570000C4948824A8AC8686946F8F732FF0948C8
:10758000428AC168084800F0CDF98FE74FF0020B3E
:1075900001E04FF0030B59460320FEF733FE00BF16
:1075A00084E700008C1300200C0400202DE9F04F2C
:1075B00099B00546002415B919B0BDE8F08F687878
:1075C000297840EA0127E878A97840EA0126012EC7
:1075D00062DB312E60DC302F5BDCB819312858DCDF
:1075E00001222046611CCCB20DF800200422204666
:1075F000611CCCB20DF800207006020E2046611C02
:10760000CCB20DF800204FF0000817E007EB08019E
:1076100088B2F9F785FA81464FEA29222046611C93
:10762000CCB20DF8002009F0FF022046611CCCB25C
:107630000DF8002008F101001FFA80F8B045E5DBE5
:1076400021466846FCF716FA82460AF0FF022046F9
:10765000611CCCB20DF800204FEA2A222046611CA2
:10766000CCB20DF800201048008AA04201DB204671
:1076700001E00D48008A0C4948824A8AC868694678
:10768000F8F7AFFE0848428AC168084800F04AF996
:1076900092E74FF0020B01E04FF0030B5946042034
:1076A000FEF7B0FD00BF87E78C1300200C0400201C
:1076B00010B5012211031448FAF76EF80122D10225
:1076C0001148FAF769F80122D1031048FAF764F873
:1076D00000224FF480410D48FAF75EF80122802124
:1076E0000A48FAF759F8012204210948FAF754F830
:1076F000012211460648FAF74FF8002210210548EA
:10770000FAF74AF810BD0000000C024000100240D9
:10771000000402400008024068480068401C6749B5
:10772000086008460068042805DD012064490860F7
:1077300000206249086063480068401C6149086095
:1077400008460068092805DD01205F49086000201F
:107750005C4908605D480068401C5C490860084658
:107760000068182805DD01205949086000205749A4
:10777000086058480068401C564908600846006880
:10778000312805DD01205449086000205149086076
:1077900052480068401C5149086008460068632848
:1077A00005DD01204E49086000204C4908604D4825
:1077B0000068401C4B49086008460068B0F5967F99
:1077C00005DB012048490860002046490860474819
:1077D0000068401C4549086008460068B0F5FA7F1B
:1077E00005DB01204249086000204049086041480B
:1077F0000068401C3F49086008460068B0F57A7F81
:1078000005DB01203C49086000203A4908603B48FC
:107810000068B0F5FA7F05DB0120394908600020D7
:107820003649086035480068401C344908603548CE
:107830000068632805DD01203349086000203149D4
:10784000086030480068401C2E4908602F480068D6
:10785000312805DD01202E49086000202B490860F1
:107860002A480068401C294908602A4800681D28E9
:1078700005DD0120284908600020264908602548C8
:107880000068401C2349086024480068B0F5FA7F6E
:107890000EDB00202149086021480068B0F5E15F57
:1078A00001DD002002E01E480068401C1C49086001
:1078B0001A480068401C194908607047F40000200D
:1078C000F0000020FC000020F8000020040100204F
:1078D000000100200C0100200801002014010020FC
:1078E000100100201C0100201801002024010020AC
:1078F000200100202C01002028010020340100205C
:10790000300100203C01002038010020440100200B
:10791000400100204C0100204801002054010020BB
:107920005001002070B504460D46164632462946E1
:107930002046FBF75FFD70BD70B50446FDF7B0FD56
:107940008020FCF7EBF82046FCF7E8F8FCF7B8F8E5
:107950000546FFF7ADFE284670BD70B505460C46DE
:10796000FDF79EFD0020FCF7D9F82846FCF7D6F875
:107970002046FCF7D3F8FFF79BFE70BD2DE9F04FD2
:107980009FB00446002500201B906078217840EAD3
:10799000012AE078A17840EA012620791D90012E85
:1079A0007EDB282E7CDC1D98C000B0427FDBBAF164
:1079B000370F79DC0AEB0600382875DC0027A9466A
:1079C0002FE009F10500205C1C904FF0000B1CE03B
:1079D000012000FA0BF01C99084018B14FF47F40C9
:1079E0001E9001E000201E900AEB070188B21E994C
:1079F000FCF7DEFC781C87B2B74202DB01201B904B
:107A000006E00BF1010000F0FF0BBBF1080FDFDB1C
:107A100000BF1B98012800D106E009F1010000F029
:107A2000FF091D988145CCDB00BF01222846691C57
:107A3000CDB201A90A540F222846691CCDB201A972
:107A40000A5401A8284421680160281DC5B22946AE
:107A500001A8FCF70FF880462846691CCDB201A9A1
:107A600001F800804FEA28222846691CCDB201A9FE
:107A70000A541348008AA84201DB284601E0104856
:107A8000008A0F4948824A8AC86801A9F8F7A9FC08
:107A90000B48428AC1680B48FFF744FF1FB001E062
:107AA00005E001E0BDE8F08F02201A9001E003201C
:107AB0001A900F201A99FEF7A5FB00BFEEE7000011
:107AC0008C1300200C0400202DE9F04F9BB00446DD
:107AD000002614B91BB0BDE8F08F6078217840EA29
:107AE0000128E078A17840EA012794F804B0012F3A
:107AF0005FDB312F5DDCBBEB470F5AD1B8F1300FA4
:107B000054DC08EB0700312850DC002512E0062089
:107B100000EB4500205C052101EB4501615C40EA7A
:107B200001201A9008EB050188B21A99FCF738FC7D
:107B3000681C85B2BD42EADB01223046711CCEB220
:107B400001A90A5410223046711CCEB201A90A5470
:107B500001A8304421680160301DC6B2314601A839
:107B6000FBF788FF81463046711CCEB201A901F8AF
:107B700000904FEA29223046711CCEB201A90A5466
:107B80001048008AB04201DB304601E00D48008A0F
:107B90000C4948824A8AC86801A9F8F722FC0948BA
:107BA000428AC1680848FFF7BDFE93E74FF0020A1A
:107BB00001E04FF0030A0AF0FF011020FEF722FB5C
:107BC00000BF87E78C1300200C0400202DE9F0474C
:107BD0009AB005468A4600246878297840EA012947
:107BE000E878A97840EA012717B1B7F57F4F43D16C
:107BF000B9F1370F3DDC39464846FCF7D9FB012285
:107C00002046611CCCB201A90A5405222046611C01
:107C1000CCB201A90A5401A8204429680160201DA2
:107C2000C4B2214601A8FBF725FF06462046611C89
:107C3000CCB201A90E5432122046611CCCB201A96B
:107C40000A541148008AA04201DB204601E00E4898
:107C5000008A0D4948824A8AC86801A9F8F7C1FB21
:107C60000948428AC1680948FFF75CFE1AB0BDE8BE
:107C7000F0874FF0020801E04FF00308414605206D
:107C8000FEF7C0FA00BFF1E78C1300200C040020BF
:107C90002DE9F0479AB005468A46002415B91AB076
:107CA000BDE8F0876878297840EA0127E878A97864
:107CB00040EA0128302F3BDC41463846FCF770FB98
:107CC00001222046611CCCB201A90A54062220469A
:107CD000611CCCB201A90A5401A8204429680160A2
:107CE000201DC4B2214601A8FBF7C4FE064620466B
:107CF000611CCCB201A90E5432122046611CCCB2D8
:107D000001A90A540E48008AA04201DB204601E086
:107D10000B48008A0A4948824A8AC86801A9F8F7CC
:107D200060FB0748428AC1680648FFF7FBFDB6E7DB
:107D30004FF0020949460620FEF764FA00BFAEE79D
:107D40008C1300200C04002010B591EA030F48BFEB
:107D500083F0004300F1C483841A71EB030C05D255
:107D6000121943EB0C03001B61EB0C01DFF824E15B
:107D70004FEA1154A4EB135C1EEA430F18BF9EEAAE
:107D8000445F73D023EA0E03DCF1200E21EA045194
:107D900043F4801332D322FA0CFE10EB0E0023FAC8
:107DA0000CFE41EB0E01CCF1200E03FA0EFE10EB9F
:107DB0000E0051F10001B1F5801FCCF1200E32D23E
:107DC00001EB045112FA0EF2BDE8104058BF7047A3
:107DD000401C38BF5FEA420218BF7047002814BF3A
:107DE00020F0010041F100014FEA410313F5001FAB
:107DF00038BF7047A1F1C04100F064BB012A43EBDA
:107E00000302ACF1200CDCF11F0E32BF4FF0000E6C
:107E100023FA0CF310EB030041EB0451B4EB115FB8
:107E2000D0D0A1EB045101F5801149085FEA300080
:107E300001EB04510ED350F1000038BF12FA0EFED0
:107E400008D1BDE81040C9E7401C38BF5FEA4202D4
:107E5000CAD1C3E7BDE810404FEA410313F5001F44
:107E600038BF7047A1F1C04100F02CBB9EEA445FCF
:107E700008D011EA5E0FBDE8104004BF01F00041D8
:107E800000207047BDE8104070B500F0CDFA00BF8B
:107E900064FBBE3E0000E0FF2DE9C04130B4DFF8D6
:107EA000A0C23CEA111418BF3CEA131400F0EC80A5
:107EB00081EA03051CEA111444EAD57418BF1CEAD0
:107EC000131500F0C780A4EB05044FF0004545EA08
:107ED000C12145EAC32341EA505143EA525304F118
:107EE0007F74994204F500344FEAC0204FEAC22261
:107EF00008BF904200F09C804FEA13650FF24016D5
:107F0000765D4FEA134506FB05F7C7F1807706FB60
:107F100007F74FEAD737A7FB03687642C8F58038E2
:107F2000A7FB06CE38BFA8F1010807FB08E64FF013
:107F3000000EA6FB028CE6FB03CEDCF1000CCEF1BA
:107F4000004E38BFAEF1010EA6FB0C584FF00007F3
:107F50004FF00005E6FB0E87A1FB08C6A0FB07CE8D
:107F600016EB0E0645F10005E1FB076515F1E04E45
:107F70007EBFA4F580345FEA46066D4116F18007A6
:107F800045F100054FEA17274FEA066647EA0567FD
:107F9000A6F1DE46B6F1805F4FEA15251FD93846B7
:107FA00024F0010C05EBC471BCF1FE6F01EB0C1168
:107FB00002D8F0BCBDE8008124425CBF01F5801E00
:107FC0009EEAC47F02D4F0BCBDE80081244238D4CC
:107FD000F0BCA1F1C041BDE8004100F073BA4FEA26
:107FE000D22242EA43524FEAD323A7FB02864FEA4A
:107FF000D02040EA415007FB03661EEA0E0F4FEA0D
:10800000D12105FB026658BFA6EB0056B6EB005621
:108010004FEA520E4EEAC37E18EB0E0E56EB530E8D
:10802000BDD518EB02085E417F1C55F10005B6E78F
:108030004FF480154FF000074FF000064FF0000896
:10804000ADE7F0BC4FF0000001F1C04101F000418C
:10805000BDE8008111EA0C1F0CEA131500D00CE0FA
:1080600013EA0C1F00F025804FF00000F0BC81EAFD
:10807000030101F00041BDE80081F0BCBDE8004112
:1080800081EA030100F01EBAF0BCBDE8004170B502
:1080900000F0CAF9097EFC3E00F007B881EA03014E
:1080A0004FF0000001F00041704781EA030100F049
:1080B00009BAF0BCBDE800414FF00000214970470B
:1080C000FFFDFBF9F7F5F4F2F0EEEDEBE9E8E6E49D
:1080D000E3E1E0DEDDDBDAD8D7D5D4D3D1D0CFCD24
:1080E000CCCBCAC8C7C6C5C4C2C1C0BFBEBDBCBB5D
:1080F000BAB9B8B7B6B5B4B3B2B1B0AFAEADACAB58
:10810000AAA9A8A8A7A6A5A4A3A3A2A1A09F9F9E31
:108110009D9C9C9B9A9999989797969595949393E3
:10812000929191908F8F8E8E8D8C8C8B8B8A89897A
:1081300088888787868585848483838282818180FD
:108140000000FF070000F87F4FEA41034FEA535356
:10815000A3F58063D3F11E03C8BFD3F1210C0CDD5E
:108160004FF0004242EAC12242EA505232FA03FC86
:108170008CEAE17CACEBE1707047102BC4BF0020AF
:10818000704703F5787CBCF1FF3F04D06FF00042EC
:1081900082EA2100704770B500F046F949922480C8
:1081A00000207047F2E700004FEA1153A3F5806307
:1081B000D3F11E03A8BFD3F1200C08DB4FF000421F
:1081C00042EAC12252EA505232FA03F070470942A1
:1081D0000BD4102BC4BF0020704703F5787CBCF192
:1081E000FF3F05D04FF0FF3070474FF00000704761
:1081F00070B500F019F900BF499224800020704743
:10820000F0E710F0004248BF4042B0FA80F310FAA5
:1082100003F10AD0C3F11D0303F580634FEA415017
:1082200002EB035202EBD12170474FF00000704780
:108230007FEAE17202D1101A62EB0101B1FA81F317
:108240000B3B24D3994012D1B0FA80F310FA03F11A
:1082500008BF7047C3F11D0303F5406303EBC2235E
:108260004FEAD1224FEA415002EB03517047C3F16C
:10827000200C20FA0CFC9840C3F1320303F5406354
:1082800003EBC22341EA0C0101EB0351704710B527
:10829000C3F1320CC3F10004C4F1200E0CF5406CA4
:1082A0000CEBC22201FA0EFC21FA04F100FA0EF3E3
:1082B000E040BDE8104040EA0C0001EB025138BF3D
:1082C0007047401C41F100015B0008BF20F0010035
:1082D00070470000DFF848C170B51CEA111E1EBFD0
:1082E0001CEA13159EEA0C0F95EA0C0F00F06F8044
:1082F00081EA030423EA4C134EEAD47E21EA4C11AE
:1083000041F4801143F48013AE44A1FB024CA0FB66
:108310000365AEF17F7E361955EB0C05A1FB034CCE
:108320004CF10003A0FB021C16EB0C06654153F157
:108330000003094218BF46F0010613F4007F0BD179
:108340004FEA03314FEA0530340341EA155140EA60
:1083500016506FF003020AE04FEAC3214FEAC5202E
:10836000F40241EA555140EA56506FF0020202EB26
:108370002E4201EB025585EACE710AD05FEA440C29
:1083800018BF24F0004450F1000041F1000120EA40
:10839000D47040F2FE7C624500D270BDA84214BF8A
:1083A0004FF080444FF04044002E08BF0024BEF13F
:1083B000806FA8BFA1F1C041BDE8704080F282800B
:1083C0004FF0000001F1C04101F0004170479EEA0A
:1083D0000C0F0CEA131518BF95EA0C0F06D04FF0DE
:1083E000000081EA030E0EF0004170BD00F01CF8A1
:1083F0008900013E00F007B800F009B84FEA430CCD
:108400005FEA5C5C08D081EA030100F05BB84FEAE8
:10841000410C5FEA5C5CF6D14FF000000149704707
:108420000000FF070000F87F0EF1020E2EF0030E91
:108430005EF8046B364205D4012A43EB030515F5BB
:10844000001F12D8012841EB010C1CF5001F0CD8AD
:108450000ED14FEAD17C15F5001F0CEB4C0C0CF142
:10846000020C08BF4CEBD37C04E04FF0080C01E099
:108470004FEAD37C0CEB4C0526FA05F606F007060E
:10848000B6F1040C06D20EEB860CBDE870404CF041
:10849000010C6047DFE80CF0090B02024FF00041CD
:1084A0004FF00000A1F5002170BD194610460128CB
:1084B00051EB010418BFD4F5001484BF002001F073
:1084C000004170BD0808A0F500114FEA3101704766
:1084D00010B591EA030F48BF83F000433FF53CAC71
:1084E000841A71EB030C07D212198CF0004C43EB89
:1084F0000C03001B61EB0C01DFF8A4E14FEA1154FF
:10850000A4EB135C1EEA430F18BF9EEA445F00F021
:10851000B08023EA6E03524221EA0451C3EB6E039A
:1085200038BF5B1EDCF1200E25D322FA0CFE10EBC7
:108530000E0043FA0CFE41EB0E01CCF1200E03FAC3
:108540000EFE10EB0E0051F10001CCF1200E29D4EB
:1085500012FA0EF201EB0451BDE8104058BF70470B
:10856000401C1CBFB2F1004F704700280CBF491CD3
:1085700020F00100704712EB020E43EB030218BF1C
:108580004FF0010E4EEA4202ACF1200CDCF11E0E5F
:1085900054D943FA0CFE10EB0E0051F1FF31CCF12F
:1085A0001E0ED5D50EF1010E12FA0EFE404141EB22
:1085B000010101EB445C5FEA5C5C10D910EBDE70FA
:1085C00001EB045138BFBEF1004FBDE8104018BFA9
:1085D000704700280CBF491C20F00100704730D2C2
:1085E0004FEAD42C11F5001124F400641BD0B1FA29
:1085F00081F20B3AA41AA41ED2F12003914030FA62
:1086000003F31943904001EBCC71002C01EB0451B2
:10861000BDE81040A8BF704701F1C0414FF0000015
:1086200001F000417047B0FA80F310FA03F100D175
:1086300010BDE41A173C4805C90AE4E701EB0451F0
:1086400010BD491001EB0451BDE810404FEA300065
:1086500002E04FF0000170474A0008BF0042F8D026
:10866000B2F5001F28BF704701F000414FF0000035
:1086700070479EEA445F07D011EA5E0FBDE81040E4
:1086800004BF002100207047BDE8104070B5FFF71F
:10869000CBFE00BF40DFF63E83F00041104670473E
:1086A0000000E0FF4FF04070E1EE100A7047000656
:1086B0001016000610160000000000000000010265
:1086C000030406070809000000000102030400007B
:1086D000F08600080000002098010000C401000896
:1086E0001087000898010020301A000020020008BE
:1086F0004132104201034D24F43954012B02D76456
:108700000510CDCC4C3D32055AFF010110329800C6
:040000050800018965
:00000001FF
